:020000040800F2
:10000000C80D002059020008BD2B000897140008F5
:10001000B92A00080D090008793A0008000000001C
:10002000000000000000000000000000293200086D
:10003000DD09000800000000552C0008F538000814
:1000400073020008730200087302000873020008BC
:1000500073020008730200087302000873020008AC
:10006000730200087302000873020008730200089C
:1000700073020008730200086D090008730200088B
:10008000730200088D09000873020008730200085B
:10009000730200087302000873020008730200086C
:1000A000730200087302000873020008730200085C
:1000B00073020008DD3900087302000873020008AB
:1000C000730200087302000873020008730200083C
:1000D000730200086D3A00086F3A0008733A00088E
:1000E000730200087302000873020008730200081C
:1000F000730200087302000873020008730200080C
:1001000073020008730200087302000873020008FB
:10011000730200087302000873020008693A0008BD
:10012000AD090008D909000873020008730200082D
:1001300073020008730200087302000873020008CB
:1001400073020008730200087302000873020008BB
:1001500073020008DB09000873020008773A000800
:10016000730200087302000873020008730200089B
:100170007302000873020008730200080000000008
:10018000730200087302000800F002F800F054F84F
:100190000AA090E8000C82448344AAF10107DA45E2
:1001A00001D100F049F8AFF2090EBAE80F0013F0E0
:1001B000010F18BFFB1A43F001031847646A0000DF
:1001C000846A00000A4410F8014B14F00F0508BFC0
:1001D00010F8015B240908BF10F8014B6D1E05D013
:1001E00010F8013B6D1E01F8013BF9D1641E03D0EC
:1001F000641E01F8015BFBD19142E4D3704700001B
:100200000023002400250026103A28BF78C1FBD81F
:10021000520728BF30C148BF0B607047632900F008
:100220003E82732900F04382002070471FB506F01C
:100230008FFB1FBD10B510BD00F078FA1146FFF717
:10024000F5FF05F0A5FA00F096FA03B4FFF7F2FF08
:1002500003BC00F097FA00000948804709480047AE
:10026000FEE7FEE7FEE7FEE7FEE7FEE7FEE7FEE766
:10027000FEE7FEE704480549054A064B70470000C3
:10028000CD39000889010008C8070020C80D0020EA
:10029000C8090020C809002053EA020C00F0698058
:1002A0002DE9F04B4FF00006002B1FBFB3FA83F58A
:1002B00003FA05F424FA05F65E4012BF1643B2FABB
:1002C00082F502FA05F4C5F120051EBF22FA05FCED
:1002D00044EA0C04203556EA044C4FEA144418BF93
:1002E000641C4FF000084FF00009904271EB030CC2
:1002F00039D3002919BFB1FA81F701FA07F6B0FA2C
:1003000080F700FA07F6C7F120071EBF20FA07FCA6
:1003100046EA0C062037B6FBF4FCA7EB0507103FB6
:1003200007F01F0BCBF120060CFA0BFB2CFA06F69C
:1003300044BFB3460026202FA4BF5E464FF0000BFB
:100340005BEA060C08BF4FF0010B19EB0B09ABFB86
:10035000027C48EB0608C01B06FB02CC0BFB03CC5F
:1003600071EB0C01C1E70B46024641464846BDE829
:10037000F08B13B54FF000004FF00001AFF3008099
:10038000BDE81C40704700000FB41CB50C0007AA64
:10039000009001D02044401E074B7B4469460190E9
:1003A000069800F052F9002C03D06946002000F0B6
:1003B0005FF91CBC5DF814FBDD0200002DE9F04183
:1003C0000E460446002020622046E168884730B38C
:1003D000252805D0D4E901219047206A401CF2E786
:1003E000E168204600278847050018D0A5F14100A4
:1003F000192802D820354FF4006732462946204696
:100400002760FFF70BFF40B1012804D0F61D26F04E
:1004100007060836D8E7361DD6E72846DAE7206A09
:10042000BDE8F08170B50C460546012A05D0287854
:10043000800600D5EA69002302E0012305E05B1C89
:10044000934202D2E05C0028F9D1A869E618C01AEC
:10045000A861286A184428622846AFF3008004E0A7
:10046000D5E9012114F8010B9047B442F8D328468E
:10047000AFF3008070BD10B5431C02E010F8011B03
:1004800071B18107FAD14FF0013202C88C1A8C4346
:1004900014EAC211F9D0C01A0A0603D0C01E10BD5A
:1004A000C01A10BD0A0401D0801E10BD0902FCD084
:1004B000401E10BD40EA010370B59B072ED14FF0DE
:1004C0000136042A2AD308C810C99D1B9D43121F58
:1004D00015EAC61517D0D8B2E1B2401A50EA056144
:1004E00010D198B2A1B2401A50EA05410AD123F0C6
:1004F0007F4024F07F41401A50EA052102D1180EB6
:10050000A0EB146070BDA342DBD018BA21BA8842B8
:1005100001D9012070BD4FF0FF3070BD0AB9002035
:1005200070BD10F8013B11F8014B63B1A3420AD131
:10053000521E08D010F8013B11F8014B1BB1A34229
:1005400001D1521EEDD1181B70BD032A40F230803C
:1005500010F0030C00F0158011F8013BBCF1020F04
:10056000624498BF11F801CB00F8013B38BF11F885
:10057000013BA2F1040298BF00F801CB38BF00F89C
:10058000013B11F0030300F09680083AC0F00880A8
:1005900051F8043B083A51F804CBA0E80810F5E7FD
:1005A000121D5CBF51F8043B40F8043BAFF30080E0
:1005B000D20724BF11F8013B11F801CB48BF11F855
:1005C000012B24BF00F8013B00F801CB48BF00F825
:1005D000012B70474FF0000200B513469446964633
:1005E000203922BFA0E80C50A0E80C50B1F1200146
:1005F000BFF4F7AF090728BFA0E80C5048BF0CC0F4
:100600005DF804EB890028BF40F8042B08BF704751
:1006100048BF20F8022B11F0804F18BF00F8012BC3
:10062000704770477047704710B500F077F8006862
:1006300010BD10B5044600F071F8046010BD000054
:1006400001694A1C02610878704700B58FB0CDE996
:1006500001310021059105497944CDE90310114686
:100660006846FFF7ABFE0FB000BD0000E5FFFFFFDF
:100670000A6802F8010B0A607047D1E900239A4228
:1006800002D2531C0B601070704710B5436913B150
:10069000AFF3008001E0FFF7C5FE012010BD127826
:1006A00000F124010A7000224A700122EDE711686E
:1006B0004FF0FF32E9E710B5203AC0F00B80B1E807
:1006C0001850203AA0E81850B1E81850A0E8185087
:1006D000BFF4F5AF5FEA027C24BFB1E81850A0E890
:1006E000185044BF18C918C0BDE810405FEA827CAA
:1006F00024BF51F8043B40F8043B08BF7047D207C1
:1007000028BF31F8023B48BF11F8012B28BF20F861
:10071000023B48BF00F8012B7047000000487047BB
:100720006407002000487047640700207546FFF703
:10073000F9FFAE4605006946534620F0070085469E
:1007400018B020B5FFF796FDBDE820404FF0000639
:100750004FF000074FF000084FF0000B21F00701A9
:10076000AC46ACE8C009ACE8C009ACE8C009ACE8EC
:10077000C0098D4670470446AFF300802046FFF75E
:1007800064FD000001491820ABBEFEE72600020010
:100790007047000030B5354D04462DED028B83B017
:1007A0000121284601F0DDF80028F9D1082C0BD2F0
:1007B000DFE804F0040650525456585A082100E06D
:1007C0001821012000F05CF8FC208DF800000A23BD
:1007D00001226946264800F09CFC00208DF80000AC
:1007E0000A2301226946224800F093FC01208DF87B
:1007F000000002460A2369461D4800F08AFC0A23CD
:10080000032201A91A4800F0D9FB9DF804009DF8C5
:100810000510000440EA01209DF80610154C08431D
:100820009FED158B20606060010205D5C043C0F3C9
:100830001600401C4042606005F0DDFC53EC182BB4
:1008400005F090FDC4E9020194ED020B03B0BDEC8C
:10085000028B30BD2821B4E73821B2E74821B0E748
:100860005821AEE76821ACE77821AAE7000C0240E6
:10087000D00100200001002085F90F270088433FA8
:1008800033B5124D81B004460121284601F069F8C4
:100890000028F9D104F00F0040F050008DF800005E
:1008A0000A23012269460A4800F033FC00208DF833
:1008B00000000A2301226946054800F02AFC0A23A9
:1008C000012202A9024800F024FC3EBD000C0240B7
:1008D000D00100200C4910B50220886106210020BB
:1008E000FFF7CEFF08210120FFF7CAFF00210220F9
:1008F000FFF7C6FF82210320FFF7C2FF0021BDE8FA
:1009000010400420FFF7BCBF000C0240FEE70000CF
:1009100070B512484FF40012531005781048941027
:100920001049092D07D2DFE805F0060507090B0E6F
:1009300010121400826170BD836170BD846170BD4E
:100940000421816170BD8A6170BD8B6170BD8C6155
:1009500070BD05498020886170BD00001C01002029
:100960000010024000040240000C024006480168EA
:10097000C1F3C061002905D04FF0006181600321FF
:1009800000F08ABE704700000060024006484168DF
:10099000C1F34051002905D04FF40011C160062178
:1009A00000F07ABE7047000000600240084801680D
:1009B000C1F3401111B1074A01211170202181605A
:1009C0000168C1F3C001002901D00821816070478E
:1009D000006402403800002070477047704772B6CC
:1009E000FEE70000024931F8100080B270470000B5
:1009F000DA000020024931F8100080B27047000090
:100A0000A80000201038C217094B00EB527210B535
:100A100003EBE20322F00702841A1B78012202FA98
:100A200004F0184201D00A7010BD0020087010BDFB
:100A3000A4000020084A10B502EBD00200F0070421
:100A40001378012202FA04F0184201D00A7010BD96
:100A50000020087010BD0000A60000202DE9F04124
:100A60002A4C00260221A220266102F05BF904F143
:100A70001005274FA878697800EB0120217827F826
:100A800011000221A420266102F04CF9A8786978AF
:100A900000EB0120217807EB410108820221A6200A
:100AA000266102F03FF9A878697800EB01202178EF
:100AB00007EB410108840221A820266102F032F9E7
:100AC000A878697800EB0120217807EB41010886BE
:100AD0000221AA20266102F025F9A878697800EBA6
:100AE0000120217807EB4101A1F840000221AC2050
:100AF000266102F017F9A878697800EB01202178C7
:100B000007EB4101A1F85000BDE8F0811C01002075
:100B10007C0600202DE9F84FDFF8BCA1002201255A
:100B200003264FF00F090AF1040BAAF1040E00BFCF
:100B30000B6805FA02F42340A34270D10F7907F045
:100B40000307012F01D0022F16D187684FEA420810
:100B500006FA08FC27EA0C07D1F80CC00CFA08FCCE
:100B60004CEA070CC0F808C04768A7430C79C4F3E7
:100B7000001494403C4344600C79E443A4070AD039
:100B8000C4684FEA420C06FA0CF7BC438F6807FAB8
:100B90000CF72743C7600C7904F00304022C12D130
:100BA000D40800EB840CDCF820405707FF0E09FA4C
:100BB00007F824EA0804D1F8108008FA07F848EA90
:100BC0000408CCF8208004684FEA420C06FA0CF7BF
:100BD000BC430F7907F0030707FA0CF727430760B8
:100BE0004C6814F4403F70D03C4C276847F4804771
:100BF0002760246822F0030704F480440094384CF2
:100C000007EB040CDCF8084897074FEA177809FA55
:100C100008F7BC43334FB84202D1002724E054E028
:100C2000314FB84201D101271EE0304FB84201D107
:100C3000022719E02E4FB84201D1032714E02D4FAF
:100C4000B84201D104270FE02B4FB84201D105274C
:100C50000AE02A4FB84201D1062705E0284FB842E2
:100C600001D1072700E0082707FA08F72743CCF847
:100C70000878DAF800405746D1F804C09C435FEA90
:100C8000CC2C00D51C433C60DBF800405F46D1F81B
:100C900004C09C435FEA8C2C00D51C433C60DEF80A
:100CA00000407746D1F804C09C435FEA8C3C00D5F5
:100CB0001C433C60084F083F3C68D1F804C09C438B
:100CC0005FEACC3C00D51C433C60521C102AFFF468
:100CD0002FAFBDE8F88F0000083C014044380240C7
:100CE00000300140000002400004024000080240C1
:100CF000000C0240001002400014024000180240A4
:100D0000001C0240014880687047000094000020E9
:100D10000248816802781144816070479400002085
:100D20000B4810B5016841F400710160016841F49D
:100D300080610160016841F480710160032000F06E
:100D400063F8002000F006F800F024F8002010BD41
:100D5000003C024070B50D4D04464FF47A7128787E
:100D6000B1FBF0F00A490968B1FBF0F000F07FFB3D
:100D700048B9102C07D200222146501E00F024F85A
:100D800000206C6070BD012070BD00009400002048
:100D9000A00000200B4882B0016841F4804101604E
:100DA000006800F4804000900648001F016841F090
:100DB00080510160006800F080500090052002B072
:100DC00000F022B844380240F0B40E4B1B680C46C9
:100DD000C3F30223C3F10705042D00D90425191D0F
:100DE000072901D2002300E0DB1E012606FA05F1E7
:100DF000491E214099409E40761E16403143F0BC6A
:100E000003F094B80CED00E0064900F00702086812
:100E10004FF6FF03184040EA0220034A10430860DF
:100E2000704700000CED00E00000FA0570B504000A
:100E300009D0606A002540B125616561A56294F81A
:100E4000510040B10CE0012070BD6068B0F5827FB8
:100E5000F4D0E561F2E784F85050204600F044F801
:100E6000022084F851002068016821F040010160EF
:100E7000A088218900F4827001F404410843A1890B
:100E800001F400610843217C01F002010843217D47
:100E900001F001010843218B01F400710843217F17
:100EA00001F03801084394F8201001F08001084354
:100EB000218D01F40051084321680860A0690421D4
:100EC00001EA104094F8241001F010010843216851
:100ED00048602068C16921F40061C1616565012035
:100EE00084F85100002070BDF0B587B0044614218D
:100EF0006846FFF76FFB2C4B226800242B49022524
:100F000003262B489A421AD1284A1432136843F414
:100F100080531360126802F4805205920A6842F00E
:100F200001020A600968029401F001010591E021C3
:100F3000CDE900150521CDE90361694630E01D4B7F
:100F40009A422FD1194A1032136843F400431360B8
:100F5000126802F4004205920A6842F001020A6037
:100F60000A6802F0010205920A6842F004020A606F
:100F7000096802AA01F0040105914FF40041CDE98E
:100F80000015062782E8D0006946FFF7C3FD4FF43D
:100F9000E050CDE9000502AA694682E8D000064883
:100FA000FFF7B8FD07B0F0BD003001403038024017
:100FB00000000240003C0040000802402DE9F84FCC
:100FC000044690F85100984616460F460025012821
:100FD00001D0022598E060684FF0040BB0F5827FE5
:100FE00001D1A068F8B194F85000012826D04FF044
:100FF000010984F85090FFF785FE8246002F7FD0CC
:10100000002E7DD084F851B000206065A763A687CC
:10101000E6872063A086E08620646064A068B0F55F
:10102000004F0DD016E084F851B013460A46204612
:10103000CDF8008000F024F9BDE8F88F0220FBE72E
:101040002068016821F0400101602068016821F4F6
:101050008041016020680168490603D4016841F0BD
:1010600040010160E068D8B13BE020688168C907B1
:1010700009D0007BA16B0870A06B401CA063E08FBF
:10108000401EE0870CE0FFF73DFEA0EB0A01414562
:1010900003D3B8F1FF3F03D006E0B8F1000F03D04F
:1010A000E08F0028E1D11FE003252BE02068816854
:1010B000C90709D0C068A16B0880A06B801CA06321
:1010C000E08F401EE0870CE0FFF71CFEA0EB0A015A
:1010D000414503D3B8F1FF3F03D0E5E7B8F1000F76
:1010E000E2D0E08F0028E1D152464146204601F08F
:1010F000DAFF08B120206065606D00E000E008B113
:10110000012501E084F85190002084F85000284621
:1011100092E72DE9F84F044690F8500000269846D3
:1011200015468A4601280CD0012784F85070FFF735
:10113000E9FD814694F85100B346012804D0022607
:101140009AE00220BDE8F88FBAF1000F6FD0002DB1
:101150006DD0032084F85100C4F854B0C4F830A016
:10116000A586E586C4F838B0A4F83CB0A4F83EB033
:10117000C4F844B0C4F840B0A068B0F5004F09D13D
:101180002068016821F0400101602068016841F495
:101190008041016020680168490603D4016841F07C
:1011A00040010160E068B0F5006F606803D058B39B
:1011B000012D29D049E008B1012D1FD1206B2168F4
:1011C0000088C86006E020688168890709D5216B1E
:1011D0000988C160206B801C2063E08E401EE08681
:1011E0000CE0FFF78FFDA0EB0901414503D3B8F1F7
:1011F000FF3F03D006E0B8F1000F03D0E08E0028D7
:10120000E1D125E0032635E0206B216800780873E2
:1012100006E02068816889070AD5216B0978017387
:10122000206B401C2063E08E401EE0860DE01FE036
:10123000FFF768FDA0EB0901414503D3B8F1FF3F7B
:1012400003D0DFE7B8F1000FDCD0E08E0028E0D15A
:101250004A464146204601F055FF08B1202060650E
:10126000A06818B92068C16880680090606D08B1F6
:10127000012601E084F8517084F850B0304661E7EF
:101280002DE9FF4F81B0044690F8500000260E9FD4
:101290001D4693464FF0010901280FD04FF0010A77
:1012A00084F850A0FFF72EFD804694F85100616845
:1012B00001280DD0B1F5827F08D103E0022005B0EE
:1012C000BDE8F08FA16809B9042801D00226C9E061
:1012D0000298002865D0BBF1000FFBD0002DF9D09B
:1012E00094F85100042802D0052084F85100002011
:1012F0006065C4F838B0E587A58702992163E58663
:10130000A5862064606420680168490603D40168EA
:1013100041F040010160E068B0F5006F606803D003
:10132000F0B3012D47D081E008B1012D3CD1206BF5
:1013300021680088C860206B801C2063E08E401EFE
:10134000E08631E02068816889070FD5E18E69B1B8
:10135000B9F1010F0AD1216B0988C160206B801C93
:101360002063E08E401EE0864FF00009206881680F
:10137000C9070CD0E18F51B1C068A16B0880A06B88
:10138000801CA063E08F401EE0874FF00109FFF74B
:10139000B9FCA0EB0800B84206D3781C04D001E0E9
:1013A00009E05BE003265BE0E08E0028CAD1E08F15
:1013B0000028C7D140E0206B216800780873206BBB
:1013C000401C2063E08E401EE0862FE0206881688C
:1013D00089070FD5E18E69B1B9F1010F0AD1216BEF
:1013E00009780173206B401C2063E08E401EE0866C
:1013F0004FF0000920688168C9070CD0E18F51B116
:10140000C068A16B0870A06B401CA063E08F401EF9
:10141000E0874FF00109FFF775FCA0EB0800B84228
:1014200002D3781C02D0BAE7002FB8D0E08E002893
:10143000CCD1E08F0028C9D142463946204601F080
:1014400061FE18B10126202060650BE0A06818B984
:101450002068C16880680090606D08B1012601E0D5
:1014600084F851A0002084F85000304627E710B5DA
:10147000401EB0F1807F01D3012010BD4FF0E02469
:1014800060610F21601702F051FD0020A06107206C
:101490002061002010BDFEE730B5134C4B680022E0
:1014A000A468124D04F00104AD6805F001052C4359
:1014B0000F4DAD6805F001052C4302D00122104606
:1014C00030BD0C4D53B10C681C43D1E902310B43C4
:1014D00041681C4329400C434460F0E743680968B5
:1014E0002B400B434360EAE700200140002101400C
:1014F00000220140E010FCFF30B58368002213F0A9
:10150000010F02D00122104630BD8C680B682343C6
:101510004468054D2C40234343608368496823F4A5
:1015200000630B438360EEE7FFFEFFFC30B54B68C2
:101530008468002214F0010F02D00122104630BD51
:10154000002B436823F4684301D08C682343436035
:10155000D1E9033423438468074D2C400D6805F01E
:1015600070652C43234383604968C36A23F4700386
:101570000B43C362E2E70000FDFCFFC010B54FF46F
:10158000407494FAA4F401F44073B4FA84F4E34090
:1015900000EB8300C36A01F01F011F248C4002F09E
:1015A0001F02A3438A401343C36210BD70B54FF0BE
:1015B000007494FAA4F401F00073B4FA84F4E340E4
:1015C00000EB8300C3684FF0F87494FAA4F501F0BF
:1015D000F871B5FA85F521FA05F50726AE4094FABB
:1015E000A4F4B4FA84F4E140B3438A401343C360E3
:1015F00070BD0000044908B50A6802430A60096822
:101600000140009108BD000030380240044908B58F
:101610000A6802430A6009680140009108BD0000A1
:1016200030380240044908B50A6802430A60096874
:101630000140009108BD000030380240044908B55F
:101640000A6802430A6009680140009108BD000071
:1016500040380240044908B50A6802430A60096834
:101660000140009108BD000040380240044908B51F
:101670000A6802430A6009680140009108BD000041
:1016800044380240034A1430515C0A5822F00402E4
:101690000A507047336B0008034A515C425822F0ED
:1016A00001024250704700002B6B0008034A515C56
:1016B000425842F01002425070470000336B00085D
:1016C000034A515C425842F0010242507047000008
:1016D000336B0008034B595C435823F0606313439A
:1016E00043507047336B0008044B001D595C0B5886
:1016F0006FF30F0313430B5070470000336B000868
:10170000034B595C435823F0C003134343507047C5
:10171000336B0008034B595C435823F48063134335
:1017200043507047336B0008034B595C435823F414
:10173000C043134343507047336B0008034B595C5D
:10174000435823F49073134343507047336B00089E
:10175000034B595C435823F40073134343507047C1
:10176000336B0008034B595C435823F4C0531343B5
:1017700043507047336B0008034B595C435823F4C4
:101780004033134343507047336B000830B5264A4B
:10179000002405790168131F85B371B345798DB1B4
:1017A000012D17D0022D18D0012483792BB31E49A7
:1017B00008310A1F012B18D0022B20D0032B22D076
:1017C000012428E015688D43156001681A680A43F2
:1017D0001A60EAE71D688D4301E01D680D431D6036
:1017E000016813680B431360DFE703680D689D43CE
:1017F0000D6000681168014311600CE00DE00368A2
:1018000015689D4302E0036815681D431560006874
:101810000A6802430A60204630BD1D688D431D6082
:10182000006811688143E7E7043C0140F0B50A68AD
:101830000F2692FAA2F2B2FA82F303248AE0012779
:101840009F4015EA07027DD04D68012D01D0022D81
:101850001BD18D68876892FAA2FCBCFA8CFC4FEA17
:101860004C0C04FA0CFC27EA0C0792FAA2FCBCFA16
:101870008CFC4FEA4C0C05FA0CF52F438760CD68C1
:101880004768554397432F4347600F69D0F80CC012
:1018900092FAA2F5B5FA85F54FEA450E04FA0EF56F
:1018A0002CEA050C92FAA2F5B5FA85F56D00AF4069
:1018B0004CEA070CC0F80CC04D68022D33D192FAE7
:1018C000A2F5B5FA85F5082D15D2D1F814C0056A30
:1018D00092FAA2F7B7FA87F7BF0006FA07F7BD43F7
:1018E00092FAA2F7B7FA87F7BF000CFA07FC45EAAD
:1018F0000C05056217E0D1F814E0476A150A95FA5D
:10190000A5FCBCFA8CFC4FEA8C0C06FA0CFC95FA90
:10191000A5F5B5FA85F5AD0027EA0C070EFA05FE28
:1019200047EA0E0747624D68076892FAA2FCBCFAC4
:101930008CFC4FEA4C0C04FA0CFE27EA0E0792FAD4
:10194000A2F200E005E0B2FA82F2520095402F4385
:1019500007605B1C0A681546DA407FF470AF002010
:10196000F0BD0069814301D000207047012070471D
:101970000069814301D0002070470120704710B5F5
:10198000044601F093F9206001F066F9606001F00F
:1019900071F9A060606801F07BF9E06010BD10B5DE
:1019A00003680122C3F380132BBBD1E900231A4340
:1019B000D1E9023423431A430B691A434B691A4392
:1019C0008B691A43CB691A430B6A1A4303684FF6B3
:1019D000BF74A3431A43026042684B6922F00402B9
:1019E00042EA134242600A6AB2F5005F02D1898C72
:1019F00089B201610022C16921F40061C161104610
:101A000010BD00000149086070470000A0000020E0
:101A100010B501291CD004291CD010291CD0402944
:101A20001CD0B1F5807F1BD0B1F5806F1AD0062194
:101A30000D4B18305B5C184403680B4CE41D615C73
:101A400003248C40120CA3438A401343036010BD4F
:101A50000021EDE70121EBE70221E9E70321E7E7B8
:101A60000421E5E70521E3E7166B000810B501291D
:101A70001CD004291CD010291CD040291CD0B1F541
:101A8000807F1BD0B1F5806F1AD006210D4B183026
:101A90005B5C184403680B4CE41D615CF0248C40D3
:101AA000120CA3438A401343036010BD0021EDE7ED
:101AB0000121EBE70221E9E70321E7E70421E5E75C
:101AC0000521E3E7166B000810B5012916D004299B
:101AD00016D0102916D0402916D0B1F5807F15D028
:101AE000B1F5806F14D00623016A0A4CE35C0A2426
:101AF0009C40A1439A401143016210BD0023F3E7CB
:101B00000123F1E70223EFE70323EDE70423EBE7EB
:101B10000523E9E7246B000810B501291CD004292E
:101B20001CD010291CD040291CD0B1F5807F1BD0BF
:101B3000B1F5806F1AD006210D4B18305B5C18444C
:101B400003680B4CE41D615C0C248C40120CA34315
:101B50008A401343036010BD0021EDE70121EBE74C
:101B60000221E9E70321E7E70421E5E70521E3E7AF
:101B7000166B0008F0B50268254B264D264E274F00
:101B8000274C4FF0804C984209D0604507D0A842BE
:101B900005D0B04203D0B84201D0A04205D1D1F85F
:101BA00004E022F0700242EA0E0298421BD0604527
:101BB00019D0A84217D0B04215D0B84213D0A042D5
:101BC00011D0184DA8420ED0174DA8420BD0174D7A
:101BD000A84208D0164DA84205D0164DA84202D002
:101BE000154DA84203D1CD6822F440722A43026009
:101BF0008A68C2620A888262984201D0A04201D1FA
:101C000009690163416941F0010141610020F0BDB2
:101C1000000001400004004000080040000C0040AB
:101C200000040140004001400044014000480140E0
:101C300000180040001C004000200040016921F411
:101C400090410161416921F02A0141617047000022
:101C500010F1140050E8001F41F0800140E800122C
:101C6000002AF7D17047000010F10C0050E8001F67
:101C700041F0200140E80012002AF7D1704700002F
:101C80007FB50446C0680D460126C0F34030C0BB96
:101C9000E9686868AA690843296911430843E1684B
:101CA00049F20C6291430843E060A868216921F47D
:101CB0004051014321616869616921F44071014328
:101CC00061616846FFF75BFE0F48844208D00F4809
:101CD00084420DD00E4884420AD00E48844201D17D
:101CE000039906E00C48844202D00C48844208D193
:101CF000029931B12B6823B100262046AA6900F071
:101D00000FF804B0304670BD0010014000440040A0
:101D10000048004000140140004C004000500040CA
:101D20002DE9F04106461920A1FB00011F460023C2
:101D300064243225B2F5004F27D0BB0FBA00FEF75E
:101D4000ABFA0146B0FBF4F06FF01802504301EB20
:101D5000800005EB0010B0FBF4F000F0F002B1FBE6
:101D6000F4F002EB0012B1FBF4F06FF018035843EB
:101D700001EB800005EB0010B0FBF4F000F00F0069
:101D8000104480B2B060BDE8F081FA195B41FEF703
:101D900083FA0146B0FBF4F00201B1FBF4F06FF0FE
:101DA0001803584301EB800005EBC000B0FBF4F0D2
:101DB00000F0F80002EB4002B1FBF4F0584301EBF5
:101DC000800005EBC000B0FBF4F000F00700D7E79F
:101DD00008B54FF0E0210A690092421C00D0401C77
:101DE0000A69D20300D5401E0028F9D108BD0000C1
:101DF00010B58EB001228DF8002040F080008DF8E3
:101E000001008DF802100321684600F056FE8DF89F
:101E100003000A4C000A8DF80400228A0520052AD6
:101E200000D3024662826946E068FEF78EFB628A52
:101E30000348E16803F072FD0EB010BD6806002093
:101E4000004800400D4910B54FF48000886101F052
:101E5000EDF90B4C0120207001F01CF9FEF7FEFD9E
:101E60000220207001F016F9FEF7F8FD0320207023
:101E700001F010F9BDE81040FEF7F0BD001002407F
:101E80001C01002030B593B000240F94109414214D
:101E900068461194FEF79EFB0B940C940D94182148
:101EA00005A80E94FEF796FB52484FF48075016822
:101EB00041F480710160006800F4807012904D4818
:101EC0001438016841F001010160006805A900F0C3
:101ED00001001290072005900320069009944648BF
:101EE000FFF7A4FC4648454902788A58037822F057
:101EF0006062CA5002788A58037822F0C002CA5041
:101F000002788A58037822F44032CA5002788A58FC
:101F1000037822F4907242F48072CA5002788A5890
:101F2000037822F40072CA5002788A58037842F487
:101F30008062CA5002788A58037822F4C05242F470
:101F40000062CA5002788A58037822F4C04242F4F0
:101F50000052CA502949027814315258007822F0B0
:101F600004024250CDE91045264D0FA90F94284692
:101F7000FFF7C2FA4FF40010CDE900404FF4407073
:101F80000294CDE9034069462846FFF7CFFAA868D6
:101F900020F48060A8604FF48030CDE90B040BA9D9
:101FA0001948FFF779FA4FF00074224621142846A9
:101FB000FFF7E4FA072221462846FFF7F7FA134C09
:101FC00040F2052122462846FFF7D8FA072221468B
:101FD0002846FFF7EBFA0E4C40F20A21224628462B
:101FE000FFF7CCFA072221462846FFF7DFFA13B0A5
:101FF00030BD00004438024000000240006402404E
:102000000E6B000800200140002301400100300257
:102010000200600210B54FF48000FFF7F7FA4FF4AA
:102020000010FFF7F3FA01F041FF0022114600F023
:10203000C6FD01460E2001F049FF0E2001F00EFF03
:1020400001F034FF0022114600F0B9FD01461120D5
:1020500001F03CFF112001F001FF01F027FF0022F9
:10206000114600F0ACFD0146382001F02FFF38206A
:1020700001F0F4FE01F01AFF0022114600F09FFD6E
:102080000146392001F022FF392001F0E7FE01F07E
:102090000DFF0022114600F092FD0146452001F09F
:1020A00015FFBDE81040452001F0D8BE2DE9F04FE6
:1020B00089B000240694182168460794FEF78AFA2E
:1020C0001020FFF797FA0420FFF794FA8020FFF71B
:1020D00091FA0120FFF78EFA0220FFF78BFA082011
:1020E000FFF788FADFF8E4B17749CBF81810DFF88A
:1020F000E4817749C8F81810DFF8DC914FF08C7153
:10210000C9F81810DFF8D8A17449CAF81810764F2A
:102110007448B8613C2000900125CDE9015469461E
:102120005846CDE90345FFF781FB4FF6C07000909C
:10213000CDE901540394694658460494FFF776FBB1
:102140004EF23E000090CDE90154039469464046AA
:102150000494FFF76BFBCDE90054694640460494B4
:10216000FFF764FB18200090CDE901540394694601
:1021700048460494FFF75AFB40F607400090CDE92B
:1021800001540394694650460494FFF74FFBA8029C
:102190000326CDE90006694604943846FFF746FB5E
:1021A0004FF462500090CDE9015469463846CDE9BC
:1021B0000345FFF73BFB4CF216000090CDE90154BC
:1021C0000394694638460494FFF730FB30020090D0
:1021D000CDE9015469464046CDE90345FFF726FBAA
:1021E00028020090CDE9015469464846CDE90345EF
:1021F000FFF71CFBF002CDE900066946049448464F
:10220000FFF714FBCDE90054694638460495FFF703
:102210000DFB38200090CDE9015469465046CDE9C8
:102220000345FFF703FB6802CDE900066946049405
:102230005046FFF7FBFA009669465846019604940B
:10224000FFF7F4FA2948D0F808184FF4704292FAD0
:10225000A2F2B2FA82F221F4704106FA02F21143BC
:10226000C0F808188DF81C504FF008088DF81D4074
:10227000CDF818808DF81E5006A8FFF787FAF86889
:1022800098FAA8F1B1FA81F1490006FA01F1884300
:1022900098FAA8F1B1FA81F1490004FA01F1084372
:1022A000F860386898FAA8F1B1FA81F149008E40D7
:1022B00098FAA8F1B1FA81F14900B0438C4020436B
:1022C000386009B0BDE8F08F0000FCFF001002404C
:1022D00000003EE3000802400000024000003F0C06
:1022E00000040240000096F8000C0240003001405B
:1022F000104810B50E4901604FF482714160002111
:102300008160C1604FF400720161C0E905121822BA
:10231000C0E90721416281620A21C162FEF786FDA0
:10232000002803D0BDE81040FEF759BB10BD0000E7
:10233000003001407801002010B592B02821684695
:10234000FEF748F918210AA8FEF744F91E4801686B
:1023500041F480410160006800F4804010901A4808
:102360001038016841F0020101600068002400F0AB
:10237000020010904FF470400A9002200B9003204E
:10238000CDE90C040520CDE90E400AA90F48FFF75E
:102390004DFA4FF48270CDE900404FF48020CDE932
:1023A000044003940A20CDE908400294069407945F
:1023B000074C69462046FFF7F2FA606820F01000EB
:1023C000606012B010BD00004038024000040240BE
:1023D00000380040104810B50E4901604FF482717A
:1023E0004160002181600122C160C0E904129204B1
:1023F00082613822C0E90721416281620A21C162FB
:10240000FEF714FD002803D0BDE81040FEF7E7BA40
:1024100010BD0000003C0040D001002010B586B087
:1024200014216846FEF7D6F80220FFF707F918488E
:1024300000680022C0F30220114600F0D9FB0146DB
:102440001D2001F053FD1D2001F015FD5320ADF8B6
:102450000000002040F2E731CDE901010D4C03906E
:1024600069462046FFF786FB206840F08000206028
:10247000A06844F207018843A060606820F0700003
:102480006060A06820F08000A06006B010BD000071
:102490000CED00E00004004030B58DB0142106A81A
:1024A000FEF798F818216846FEF794F80420FFF725
:1024B000C5F83A48016841F0020101600068002453
:1024C00000F002000B904FF4E07000900220CDE984
:1024D0000104CDE90440694603943148FFF7A6F9A9
:1024E000ADF818404FF6FF70CDE9074009942D4C28
:1024F00006A92046FFF73EFB206820F08000206000
:10250000A06820F0070040F00300A060A5132A4651
:1025100001212046FFF77CFA002201212046FFF727
:10252000FBFA002201212046FFF7A0FA0022012138
:102530002046FFF7C9FA2A4610212046FFF768FA1D
:10254000002210212046FFF7E7FA00221021204642
:10255000FFF78CFA002210212046FFF7B5FA6068D9
:1025600020F070006060A06820F08000A0602A4623
:10257000A51529462046FFF74BFA0022294620469A
:10258000FFF7CAFA002229462046FFF76FFA002219
:1025900029462046FFF798FA0DB030BD303802408A
:1025A000000402400008004010B586B014216846BF
:1025B000FEF710F82020FFF741F8154800680122C7
:1025C000C0F30220022100F013FB0146372001F086
:1025D0008DFC372001F04FFC44F29F10ADF8000055
:1025E0000020019027200B4C029069462046FFF7FF
:1025F000C1FA206840F080002060606820F0700020
:102600006060A06820F08000A06006B010BD0000EF
:102610000CED00E0001400402DE9F0418EB01C21CB
:1026200006A8FDF7D7FF18216846FDF7D3FF102055
:10263000FFF71CF80120FEF7F5FF4FF400700225AC
:102640000024CDE9000503260727CDE90264DFF861
:102650007080CDE9044769464046FFF7E7F8680215
:102660008DE8610001200597CDE9034069464046A9
:10267000FFF7DCF801F022FC0022114600F0D1FA4D
:102680000146252001F042FC252001F001FC4FF419
:10269000E130CDE906040C200894CDE909400B9403
:1026A0000C94084C06A92046FFF7EAFA2046FFF7EB
:1026B000C5FAE06840F40050E0600EB0BDE8F0817B
:1026C00000000240001001402DE9F0418EB01C21B5
:1026D00006A8FDF77FFF18216846FDF77BFF4FF442
:1026E0000030FEF7B7FF0820FEF79CFF20200226EF
:1026F0000024CDE9000603250727CDE90254DFF8C1
:10270000D080CDE9044769464046FFF78FF8402066
:10271000CDE90006029501200597CDE90340694601
:102720004046FFF783F82B4DB20606212846FEF7F8
:10273000D1FF402206212846FEF7E2FF00220621B3
:102740002846FFF719F8AA1506212846FEF7F6FFD6
:10275000002206212846FEF7FBFF2A1506212846FF
:10276000FEF7D8FF002206212846FEF7FBFF0022D5
:1027700006212846FEF7D8FF06212846FEF782FFED
:1027800001F09CFB0022114600F04BFA0146262086
:1027900001F0BCFB262001F07BFB4FF41640CDE995
:1027A00006040C200894CDE909400B940C940A4CC3
:1027B00006A92046FFF764FA2046FFF73FFAE068D3
:1027C00040F40050E06003F037FA0EB0BDE8F0814D
:1027D000000C024000600240004400402DE9F0413E
:1027E0008EB01C2106A8FDF7F5FE18216846FDF7FE
:1027F000F1FE4FF48020FEF72DFF0820FEF712FFB8
:102800004FF4807002250024CDE900050326072738
:10281000CDE90264DFF8E480CDE90447694640462B
:10282000FFF704F828028DE8610001200597CDE943
:10283000034069464046FEF7F9FFAA06304D0321E2
:102840002846FEF747FF402203212846FEF758FF9F
:10285000002203212846FEF78FFF0022032128468D
:10286000FEF76CFF002203212846FEF771FF2A15B0
:1028700003212846FEF74EFF002203212846FEF7DB
:1028800071FF002203212846FEF74EFF0321284650
:10289000FEF7F8FE01F012FB0022114600F0C1F92C
:1028A0000146272001F032FB272001F0F1FA4FF416
:1028B000E130CDE906040C200894CDE909400B94E1
:1028C0000C94104C06A92046FFF7DAF92046FFF7D2
:1028D000B5F9E06840F40050E0600B49084A201D5B
:1028E000C978083288502046FFF7B2F903212846FC
:1028F000FEF7DCFE0EB0BDE8F0810000000C0240E7
:102900000060024000480040336B00082DE9F041B0
:102910008EB01C2106A8FDF75DFE18216846FDF764
:1029200059FE2020FEF7A2FE0420FEF77BFE402089
:1029300002250024CDE9000503260827CDE902641D
:10294000DFF86081CDE9044769464046FEF76EFF37
:1029500080208DE8610001200597CDE9034069469C
:102960004046FEF763FF504D4FF02066324601218E
:102970002846FEF7AFFE002201212846FEF7C0FEE2
:10298000002201212846FEF7F7FEAF153A46012145
:102990002846FEF7D3FE002201212846FEF7D8FE86
:1029A0004FF48068424601212846FEF7B3FE00221C
:1029B00001212846FEF7D6FE002201212846FEF717
:1029C000B3FE01212846FEF75DFE32460621284669
:1029D000FEF780FE402206212846FEF791FE0022E7
:1029E00006212846FEF7C8FE3A4606212846FEF78D
:1029F000A5FE002206212846FEF7AAFE4246062131
:102A00002846FEF787FE002206212846FEF7AAFE8A
:102A1000002206212846FEF787FE06212846FEF7FB
:102A200031FE01F04BFA0022114600F0FAF801469F
:102A3000472001F06BFA472001F02AFA4FF41650B4
:102A4000CDE906040C200894CDE909400B940C94C0
:102A5000164C06A92046FFF713F92046FFF7EEF8BB
:102A6000E06840F40050E06004F10C0050E8001F02
:102A700041F0100140E80012002AF7D10C490B4840
:102A8000094A001D8979083288502046FFF7E0F88E
:102A900006212846FEF70AFE0648FFF7E5F80EB0C5
:102AA000BDE8F081000802400064024000140140CB
:102AB000336B000800440040FEE730B503004FF6DA
:102AC000FF7014D0814212D04AF20104491E89B22B
:102AD0000DD313F8012B50400022C5074FEA5000D8
:102AE00000D06040521CD2B2082AF6D3EEE730BDC7
:102AF00030B4002848D0022946D304784278012C0B
:102B0000134601D0002C3FD1891E052A37D008DC9E
:102B1000012A11D0022A14D0032A17D0042A06D180
:102B200019E0062A1CD00F2A1FD0102A22D030BC50
:102B300001211846FFF75CB930BC89B2801C00F057
:102B400019B930BC89B2801C00F08AB930BC89B296
:102B5000801C00F0F7B930BC89B2801C00F046BA86
:102B600030BC89B2801C01F0E1B830BC89B2801C55
:102B700000F0B0BF30BC89B2801C01F023B830BC7B
:102B800089B2801C01F094B830BC704770B50A4C13
:102B9000E188206802290ED34218891E32F8025CAF
:102BA00089B2FFF78AFF854205D1E1882068BDE838
:102BB0007040FFF79DBF70BD68060020FEE730B58E
:102BC00000F00703C3F10704042C00D90424181DE6
:102BD000072801D2002300E0DB1E012505FA04F0DE
:102BE000401E084098409D406D1E1540284330BD52
:102BF00030B500F00703C3F10704042C00D9042406
:102C0000181D072801D2002300E0DB1E012505FA6C
:102C100004F0401E084098409D406D1E154028431A
:102C200030BD30B500F00703C3F10704042C00D910
:102C30000424181D072801D2002300E0DB1E012513
:102C400005FA04F0401E084098409D406D1E154056
:102C5000284330BD7047000004490968044A01F068
:102C6000F0010909515CC840704700000838024073
:102C70003B6B000804490968044A01F4E05102EB87
:102C800091210978C8407047083802404B6B000812
:102C900004490968044A01F4604102EB51310978A2
:102CA000C8407047083802404B6B0008074800686E
:102CB00010F00C01064807D0042904D0082903D1DC
:102CC000082000F009B803487047000008380240A7
:102CD0000024F40000127A0010B5104A04460020C7
:102CE000116811F480030E4903D0B3F5800F00D1B1
:102CF0004910082C11D1106800F03F00B1FBF0F032
:102D00001168C1F3881148431168012201F4403170
:102D100002EB11414900B0FBF1F010BD0438024054
:102D20000024F40038B50C4610490022CA600C316A
:102D30000870FDF7EDFD0120FFF74AF80B4A64200B
:102D400010320090631C111F0948FEF799FA30B148
:102D500000F06CFA0120FFF73BF8012038BD00F0CD
:102D600065FA0120FFF734F8002038BD1C0100206F
:102D7000780100202DE9F04F8FB0044600200E901E
:102D800034216846FDF726FC208890FA90F8608888
:102D9000B8F11F0F47BA59D807EB0800202855D8BB
:102DA000F81DC0F3C70901208DF8000003248DF839
:102DB000010000258DF80290AA46EB4625E000218F
:102DC0000BF804104FEA010608EB050080B20DA9CC
:102DD000FDF718FE9DF834201BF80410B240114393
:102DE0006D1CADB20BF80410BD4202D3641CE4B2FA
:102DF0000DE0761CF6B2082EE6D3641C0E98E4B201
:102E000028B90AF1010000F0FF0ACA45D7D32146CC
:102E10006846FFF752FE0BF80400641CE1B2000A9A
:102E20000D4C0BF80100491C208ACAB2904200D216
:102E3000024662826946E068FDF787FB628A0748BE
:102E4000E16802F06BFD0FB0BDE8F08F02210120B8
:102E5000FEF7CEFFF7E700006806002000480040BC
:102E60002DE9F04F8FB000210E910188408891FA32
:102E700091F847BAB8F10F0F5AD807EB080010289D
:102E800056D8F81DC0F3C70901208DF800000220B4
:102E900003248DF8010000258DF80290AA46EB4628
:102EA00025E000210BF804104FEA010608EB0500AD
:102EB00080B20DA9FDF7BEFD9DF834201BF804106B
:102EC000B24011436D1CADB20BF80410BD4202D3E9
:102ED000641CE4B20DE0761CF6B2082EE6D3641C46
:102EE0000E98E4B228B90AF1010000F0FF0ACA45C1
:102EF000D7D321466846FFF7E0FD0BF80400641CB9
:102F0000E1B2000A0D4C0BF80100491C208ACAB23C
:102F1000904200D2024662826946E068FDF715FBE6
:102F2000628A0748E16802F0F9FC0FB0BDE8F08F53
:102F300002210846FEF75CFFF7E700006806002064
:102F40000048004070B58EB0002841D0018840880C
:102F50004EBA42BA501E0F283ED80F2E3AD8B0189B
:102F6000102837D801208DF8000003208DF80100CB
:102F7000500003246D468DF8020000230CE0F01889
:102F800080B2FDF72FFD010A2955641CE1B2685497
:102F9000491C5B1CCCB29BB29342F0D321466846DD
:102FA000FFF78BFD2855641CE1B2000A0D4C6854F4
:102FB000491C208ACAB2904200D202466282694607
:102FC000E068FDF7C2FA628A0748E16802F0A6FCF1
:102FD0000EB070BD022100E003210320FEF708FFC0
:102FE000F6E70000680600200048004070B58EB08B
:102FF000002841D0018840884EBA42BA501E182895
:103000003ED8182E3AD8B018192837D801208DF894
:10301000000004208DF80100500003246D468DF857
:10302000020000230CE0F01880B2FDF7E3FC010A77
:103030002955641CE1B26854491C5B1CCCB29BB29C
:103040009342F0D321466846FFF737FD2855641CAC
:10305000E1B2000A0D4C6854491C208ACAB2904261
:1030600000D2024662826946E068FDF76EFA628A23
:103070000748E16802F052FC0EB070BD022100E08A
:1030800003210420FEF7B4FEF6E7000068060020E6
:103090000048004010B51E2000F0F0FCBDE81040D4
:1030A0000320FEF795BEF8B5044640684FF48273DE
:1030B000984221D1A0684FF48065B0F5004F01D04F
:1030C000A8420AD12068066826F0400606606068BB
:1030D000984211D1A068A8420ED000920B4600225F
:1030E0008021204600F044F8002804D0606D40F0B4
:1030F000200060650320F8BD00920B4600220121EC
:10310000EFE70000F8B515460E460B460092044660
:103110000122022100F02CF8A0B9134813490068DD
:10312000B0FBF1F04FF47A71484300906068B0F55D
:10313000827F0DD13346002280212046009500F089
:1031400017F870B1606D40F0200060650320F8BD95
:10315000009830B1401E009020688068C04300068F
:10316000F6D50020F8BD0000A000002000366E015A
:103170002DE9F8431E46914688460446089DFDF712
:10318000C1FD401B351AFDF7BDFD07462548006807
:10319000C0F3CB30684338E0701C37D0FDF7B2FD88
:1031A000C01BA84203D215B1009860B32CE0206880
:1031B000416821F0E00141606068B0F5827F0BD189
:1031C000A068B0F5004F02D0B0F5806F04D1206840
:1031D000016821F040010160A06AB0F5005F09D1EB
:1031E0002068016821F4005101602068016841F401
:1031F00000510160012084F85100002084F8500043
:103200000320BDE8F8830025401E009020688168F7
:1032100038EA010004D000214945BDD10020F0E783
:103220000121F9E7A0000020704700000948202193
:1032300081611021816108218161C9038161064892
:1032400020218161102181610821816108050349E4
:10325000886170470010024000040240000C0240E8
:103260002DE9F04F48202DED0C8B83B000F006FCCB
:103270000A20FEF7ADFD03210020FFF753FDFD4CB2
:10328000E07803F020F841EC1A0B9FEDFBCBB0EE99
:103290004C1AF0EE6C1A9FEDFABBB0EE4B0AF0EE52
:1032A0006B0A00F055FEB0EE408AF0EE608AA0781E
:1032B00003F009F853EC182B03F054F841EC190B08
:1032C0009FEDF1DBB0EE4B0AF0EE6B0AB0EE4D1A5B
:1032D000F0EE6D1A00F03CFEB0EE408AF0EE608A2F
:1032E000607802F0F0FF53EC182B03F03BF853EC3E
:1032F000192B02F00FFD53EC1A2B02F00BFD02F01C
:103300004DFF0290582000F0B9FB0A20FEF760FD47
:1033100003210020FFF706FDE07802F0D4FF41EC26
:10332000190BB0EE4C1AF0EE6C1AB0EE4B0AF0EE40
:103330006B0A00F00DFEB0EE408AF0EE608AA078D5
:1033400002F0C1FF53EC182B03F00CF841EC180B02
:10335000B0EE4D1AF0EE6D1AB0EE4B0AF0EE6B0ABD
:1033600000F0F6FDB0EE40AAF0EE60AA607802F040
:10337000AAFF53EC1A2B02F0F5FF53EC182B02F0C6
:10338000C9FC53EC192B02F0C5FC02F007FF044600
:10339000B0EE4C1AF0EE6C1AB0EE4B0AF0EE6B0A7F
:1033A00000F0D6FDB34DBA4E103DB0EE408A2878FD
:1033B000F0EE608A06EB4000B0F8400002F083FFB8
:1033C00053EC182B02F0CEFF41EC180B204602F014
:1033D0007AFF53EC182B03F0D1F902F0AFFE4FF057
:1033E00080710446884201DD0C4603E0A94884420E
:1033F00000DA04469FEDA81BB0EE4B8AF0EE6B8A14
:10340000B0EE480AF0EE680A00F0A2FD2878B0EEAF
:10341000409A06EB4000F0EE609AB0F85030B346A8
:10342000A3FB04074FF0000808FB04714FEAE4799E
:1034300003FB091102F0F6FE53EC192B02F026FDF6
:103440009FED971B53EC112B02F064FC02F076FE0B
:1034500007469FED959BB0EE480AF0EE680AB0EE85
:10346000491AF0EE691A00F073FD2878B0EE40AA10
:1034700006EB4000F0EE60AA038EA3FB040C08FBF1
:1034800004C103FB091102F0CDFE53EC1A2B02F02C
:10349000FDFC41EC1A0BB0EE4D1AF0EE6D1AB0EED9
:1034A000480AF0EE680A00F053FD2878B0EE40BA02
:1034B00006EB4000F0EE60BA008A02F004FF53EC25
:1034C0001B2B02F04FFF53EC1A2B02F023FC03F0EE
:1034D00045FA774A0E4680460B21101AB14102DAAE
:1034E00010460B2608E07349B8EB010056F10700BF
:1034F00003DA08466FF007068046B0EE4C1AF0EE8D
:103500006C1AB0EE480AF0EE680A00F021FD594D41
:10351000B0EE401A103DF0EE601A2978B0EE41AAE4
:103520000BEB4100F0EE61AA018C0022A1FB040C20
:1035300002FB04C201FB092102F074FE53EC1A2BBA
:1035400002F0A4FC41EC1A0B9FED5BCBB0EE480AF5
:10355000F0EE680AB0EE4C1AF0EE6C1A00F0F8FCCF
:103560002978B0EE40BAF0EE60BA3BF8110002F0F4
:10357000AAFE53EC1B2B02F0F5FE53EC1A2B02F0C3
:10358000C9FB03F0EBF94E4B81460322181A0D4696
:103590008A4102DA1846032508E04A49B9EB0100DE
:1035A00055F1010003DA08466FF00105814600BFBE
:1035B0004FF0000A9FED44BBB7F5FA6F59DA9FED63
:1035C000441BB0EE480AF0EE680A00F0C1FCB0EE11
:1035D00040DAF0EE60DA204602F00DFE41EC100B0E
:1035E000B0EE481AF0EE681A00F0B2FC9FED3AAB6C
:1035F00051EC100B53EC1A2B02F0B4FE53EC1D2BC4
:1036000002F044FC02F09AFD83469FED351BB0EEBC
:10361000480AF0EE680A00F09BFCB0EE40DAF0EEEB
:1036200060DAA7F5FA6002F0E6FD824641EC100B85
:10363000B0EE481AF0EE681A009100F089FC53ECE5
:103640001A2B51EC100B02F08DFE53EC1D2B02F0E7
:103650001DFC02F073FD0446B0EE4A1AF0EE6A1A41
:10366000B0EE480AF0EE680A00F072FCB0EE40AA34
:103670003AE098E02C01002000000000000020400B
:10368000000000000000004000000000000030408A
:103690007C060020000100FF000000000000374011
:1036A0000000000000409F400000000000001C409F
:1036B0000000F4FFF8FF0F000000000000002E40A3
:1036C0000000FCFFFEFF03000000000000001040AF
:1036D00000000000008040400000000000000840A2
:1036E000000000000000F03F0099F0EE60AA41ECFD
:1036F00010ABB0EE481AF0EE681A00F029FC9FED0E
:10370000761B51EC100B53EC112B02F02BFE53ECFB
:103710001A2B02F0BBFB02F011FD824640F2DC5096
:10372000C7423FDA07F2DC5002F065FDB0EE48AA6E
:10373000F0EE68AACDE9000141EC100BB0EE4A1A98
:10374000F0EE6A1A00F004FC53EC192B51EC100B4C
:1037500002F008FE41EC190B204602F04CFD53EC40
:10376000192B02F0D7FA02F0E9FC0446DDE900016A
:1037700041EC100BB0EE4A1AF0EE6A1A00F0E8FBCA
:1037800053EC1B2B51EC100B02F0ECFD41EC190B30
:10379000504602F030FD53EC192B02F0BBFA02F058
:1037A000CDFC82464AE09FED4E1BB0EE480AF0EE9B
:1037B000680A00F0CDFBB0EE40AAF0EE60AA204609
:1037C00002F019FD41EC100BB0EE481AF0EE681A49
:1037D00000F0BEFB53EC192B51EC100B02F0C2FDB4
:1037E00053EC1A2B02F052FB02F0A8FC8346B0EE19
:1037F0004B1AF0EE6B1AB0EE480AF0EE680A00F0D1
:10380000A7FBB0EE401AF0EE601AB0EE419AF0EE6F
:10381000619AA7F5FA6002F0EEFC41EC100BB0EEF5
:10382000481AF0EE681A00F093FB53EC192B51EC98
:10383000100B02F02BFB02F081FC0446A7EB0B01FE
:10384000DFF8A4B0CBF80410B8EB040766EBE4761D
:10385000B9EB0A0465EBEA75B0EE4C1AF0EE6C1A9F
:10386000B0EE480AF0EE680A00F072FBB0EE40AA33
:10387000F0EE60AA3846314602F0D4FC41EC190B58
:103880009FED1A1BB0EE480AF0EE680A00F060FBEC
:1038900002990022A4FB010305FB013104FB021184
:1038A000B0EE408AF0EE608A02F0BCFC53EC182BBC
:1038B00002F0ECFA53EC192B02F060FF53EC1A2BD8
:1038C00002F0E4FA02F03AFCCBF8080000BF03B0C3
:1038D000BDEC0C8BBDE8F08F000000000000144030
:1038E00000000000008042401C0100200000000099
:1038F00000003540FDF70CBA70B52E48016821F084
:10390000070141F005010160016801F00701052987
:10391000FAD12949086840F48040086027480268C5
:1039200042F4803202600268C2F34042002AFAD0B8
:10393000224A234B121D1468224D2C40234313604E
:10394000136823F440331360026842F0807202600F
:103950000268C2F34062002AFAD04868C0F380309F
:103960000028FAD015480830016821F0F001016004
:10397000016821F4E05141F4A0510160016821F493
:10398000604141F400410160016821F0030141F010
:1039900002010160016801F00C010829FAD10A480E
:1039A000FEF730F80020FDF7D5F9002801D072B6F7
:1039B000FEE770BD003C024000700040003802404D
:1039C000042A40000080BFFF007A030A0248016811
:1039D00041F470010160704788ED00E0204B10B5A4
:1039E000186910F0010F39D01E48002101224468E7
:1039F000641C4460042C01DDC0E90021C468641C1F
:103A0000C460092C01DDC0E902214469641C4461E1
:103A1000092C01DDC0E90421C469641CC461632C64
:103A200001DDC0E90621446A641C4462B4F5967F56
:103A300001DBC0E90821C46A641CC462B4F5FA7FE2
:103A400001DBC0E90A21446B641C4463B4F57A7F4E
:103A500001DBC0E90C216FF00100186110BD00000E
:103A6000000400405400002001F06EBF704701F0D8
:103A700009BE01F013BF7047FEE70000134910B5FF
:103A80000022CA600C310870FCF742FF0120FEF7EB
:103A90009FF90E490A2301220C310D48FDF739FB2D
:103AA00000284FF00A0008D0FEF792F9FFF7BEFB9E
:103AB0000120FEF78DF9012010BDFEF789F9FFF70F
:103AC000B5FB0120FEF784F9002010BD1C01002089
:103AD000780100202DE9F04F8FB0804600200D9036
:103AE0000E90B8F8000098F804A047BAB8F80200A1
:103AF00046BA701E0F285BD8B6EBCA0F58D81F2FD6
:103B000054D8B819202851D8002420461FE000BFFF
:103B100008EB0900002590F805B00120A84010EA44
:103B20000B0F02D04FF47F4100E00021381980B222
:103B300000F0A2F8641CA4B2B4420BD26D1CEDB22A
:103B4000082DEAD30E9828B909F10100C0B28146C8
:103B50005045DDD30D9901206D460DF801000D9CF7
:103B60000F20641C0DF80400641C0DEB0401D8F850
:103B700000000860241D21466846FEF79EFF285578
:103B8000641C000A28550D4D621C288A904200D200
:103B900002466A826946E868FCF7D7FC6A8A0848E8
:103BA000E96801F0BBFE0FB0BDE8F08F022100E034
:103BB00003210F20FEF71CF9F5E70000680600203E
:103BC00000480040F0B500248DB0002845D00188A1
:103BD0004DBA41884ABA0179531E0F2B41D8B1EB37
:103BE000420F3ED10F2D3AD8A918102937D80023FB
:103BF0001E4F0AE000EB4301EE18B1F80510B6B213
:103C000049BA5B1C27F816109BB29342F2D30121EC
:103C10000DF80410641C10210DF80410641C0DEB49
:103C2000040100680860241D6D4621466846FEF7C1
:103C300044FF2855641C000A28550D4D621C288A33
:103C4000904200D202466A826946E868FCF77DFC31
:103C50006A8A0848E96801F061FE0DB0F0BD0221F2
:103C600000E003211020FEF7C3F8F6E7DA00002099
:103C700068060020004800401038C21700EB52735D
:103C800023F0070210B5801A0122084C824004EB91
:103C9000E300B1F57F4F05D0002902D101789143AF
:103CA000017010BD01781143FAE70000A400002064
:103CB00010B50446008861888EB040BA49BA41B157
:103CC000B1F57F4F05D003210520FEF791F80EB026
:103CD00010BD1F2824D8FFF7CFFF01208DF800006A
:103CE00005208DF801002068CDF802000621684605
:103CF000FEF7E3FE8DF806000A4C000A8DF8070077
:103D0000228A0820082A00D3024662826946E068B7
:103D1000FCF71BFC628A0448E16801F0FFFDD6E76E
:103D20000221D1E7680600200048004010B58EB09F
:103D3000002829D00188428849BA52BA0F2925D8CB
:103D4000154B23F8112001218DF8001006218DF864
:103D500001100068CDF802006846FEF7AEFE8DF84F
:103D600006000E4C000A8DF80700228A0820082A57
:103D700000D3024662826946E068FCF7E6FB628A8D
:103D80000748E16801F0CAFD0EB010BD022106200F
:103D9000FEF72EF8F8E70000DA00002068060020A1
:103DA0000048004004484FF40031816104218161E2
:103DB0000821816170470000000802402DE9F041B0
:103DC000194D4FF480200024A861012001F002FB6E
:103DD0000420A861012001F0FDFA01212846FDF729
:103DE000C7FD012800D1012400264FF400276400FC
:103DF000AF610A2001F00AFB0820A861052001F04C
:103E000005FB01212846FDF7B3FD012801D144F04F
:103E10000104052001F0FAFA761CF6B20F2EE6D363
:103E2000A0B2BDE8F08100000008024003B4019890
:103E30004100009850EAC12018BF04204A0D18BF65
:103E400040F0010040F2FF72B2EB515F08BF40F05A
:103E50000200012808BF052002B07047002809DBD6
:103E600000F01F02012191404009800000F1E02094
:103E7000C0F800117047002809DB00F01F02012183
:103E800091404009800000F1E020C0F80011704727
:103E9000002809DB00F01F02012191404009800049
:103EA00000F1E020C0F800117047000002480068EF
:103EB000C0F30220704700000CED00E002480068EB
:103EC000C0F30220704700000CED00E00907090E66
:103ED000002804DB00F1E02080F80014704700F0B7
:103EE0000F0000F1E02080F8141D70470907090E4B
:103EF000002804DB00F1E02080F80014704700F097
:103F00000F0000F1E02080F8141D70470907090E2A
:103F1000002804DB00F1E02080F80014704700F076
:103F20000F0000F1E02080F8141D70470907090E0A
:103F3000002804DB00F1E02080F80014704700F056
:103F40000F0000F1E02080F8141D70470000000011
:103F50002DE9F04D2DED040B2DED0C8B96B0DDE928
:103F60002350259CDDF888A025F0004624F0004869
:103F7000BAF1000F14BF0121002101EB4502FE49F7
:103F800053184A1093422AD3002814BF0123002358
:103F900003EB44030B44F9498B4220D358EA000158
:103FA0009FEDF78B6FD0DFF8E0B35D4503D1BAF139
:103FB000000F05D187E0BAF1000F08BF002100D043
:103FC000012101EB450111F5001F08D8002814BF9D
:103FD0000121002101EB440111F5001F0BD99DEDDA
:103FE000241B9DED220B16B0BDEC0C8B04B0BDE87C
:103FF000F04D00F05DBE0027002DBCBFE3498845B1
:1040000021DAE3498845A8BF02271CDAC3451ADC38
:10401000E04901EB2851142908DDC1F1340220FAEE
:1040200002F101FA02F282420DD108E058B9C1F161
:10403000140228FA02F101FA02F2424503D101F01A
:104040000101C1F1020756EA0A011DD1002C1BDA59
:10405000002D18BF022F01D0012F0AD00220FCF73B
:10406000E8FA16B0BDEC0C8B04B0BDE8F04D00F0E2
:1040700007BE0220FCF7DDFA00F002FE51EC100B47
:1040800001F03CFE83E01EE09FEDC39B9FEDC4ABBF
:10409000002872D1BD4880452DD105F1804010F532
:1040A000801008BFBAF1000F0DD0B34515DC002C0D
:1040B000A1BF9DED240B16B0BDEC0C8B04B0A8BFC6
:1040C000BDE8F08D12E0B0EE480AF0EE680A16B0D6
:1040D000BDEC0C8B04B0BDE8F08D002C06DA9DED34
:1040E000240B51EC100B01F009FE50E0AE4878446F
:1040F00090ED000BEBE7D8454FD1002C4ADA2EB1FA
:1041000086423BD1BAF1000F44D126E0BAF1000F4C
:1041100013D00220FCF78DFA00F0E6FD8DED020BC6
:104120009DED220B8DED000B10EE900A039961F3CB
:104130001E0003909DED020BC9E78DED029B9DEDE6
:10414000220B19EE901A10EE900A8DED000B61F320
:104150001E0003909DED020BB9E78DED02AB9DEDC6
:10416000220B1AEE901A10EE900A8DED000B61F3FF
:104170001E0003909DED020BA9E729E00ADA9DEDF0
:10418000220B51EC180B53EC102B01F07FFE41EC8D
:10419000100B9CE79DED220B99E7864218DAB4F1EB
:1041A000804F0DD0A4F10050B0F1FF5010D1002D80
:1041B0000EDB9DED220B51EC100B01F034FCE6E719
:1041C0009DED220B53EC102B51EC100B00F0AEBC0C
:1041D0009DED220B51EC100B01F034F9BAF1000FF8
:1041E000CDE90C0134D19FED720BDEB1A6F1E040B8
:1041F000B0F17F602CD1002D01DD002C0DDA002DF7
:1042000001DD002C1FDB002D16DA002C14DB012F42
:1042100008BF9FED690B3FF45AAFB0EE490AF0EECC
:10422000690A54E7022F18BF002D0CD0012F0AD1C4
:10423000002DFFF64CAF06E0002DB8BF002C07DACA
:10424000012F3FF444AFB0EE4A0AF0EE6A0A3EE7AF
:10425000012000EBE57A5AEA07000CD05848002507
:1042600080457CDD57495848884514DDB0420DDB58
:10427000002C19DB2BE00120FCF7DBF916B0BDECBC
:104280000C8B04B0BDE8F04D00F01EBDB34502DC60
:10429000002C09DC1BE0864202DA002C17DA03E06E
:1042A0005E4527DD002C12DD0220FCF7C2F900F08C
:1042B0001BFD10EE901A19EE900A8DED020B8DED9C
:1042C000009B61F31E0003909DED020BFFE60220B0
:1042D000FCF7AFF900F018FD10EE901A18EE900AF6
:1042E0008DED020B8DED008B61F31E0003909DEDB3
:1042F000020BECE69DED220B53EC182B51EC100B4E
:1043000002F03CFA9FED320BCDE90A0153EC102B81
:104310009DED0A0B51EC100B02F024F89FED2E1BC3
:1043200053EC112B02F052F99DED0A1B53EC112BAB
:1043300002F018F89FED2A1B53EC112B02F046F9FE
:104340009DED0A0B41EC190B53EC102B51EC100BAB
:1043500002F008F853EC192B02F004F800E07EE0BC
:104360009FED210B41EC1A0B53EC102B9DED0A0B2A
:1043700051EC100B3CE00000FFFF1F00FFFF0F009F
:10438000000000000000F03F0000F03F0000F07F60
:104390000000404301FCFFFF000000000000F07F30
:1043A0000000000000000000262B000000000000BC
:1043B0000000000000000080000000000000F0FF8E
:1043C0000000E0410000F043FFFFEF3F000000006D
:1043D000000000000000D03F555555555555D53FBC
:1043E000000000000000E03F000000604715F73FBC
:1043F00001F0B8FF41EC190B9FEDFD0B51EC1A0BCE
:1044000053EC102B01F0AEFF41EC1A0B9FEDFA0BB1
:1044100053EC102B9DED0A0B51EC100B01F0A2FF99
:1044200053EC1A2B02F0AAF941EC1A0B51EC190BC0
:1044300053EC1A2B01F06EFC0690CDE906519DED70
:10444000060B53EC192B51EC100B02F097F953ECBF
:104450001A2B02F0BBF841EC100B00F09FB90020C2
:10446000B6F5801F0EDA9FEDE60B53EC102B9DED99
:104470000C0B51EC100B01F075FFCDE90C016FF046
:1044800034000E4600EB2650A0F2FF38C6F31300AE
:10449000DD4940F07F6646F040568842D8BF002490
:1044A00009DDDA498142C8BF012404DC0024A6F5F5
:1044B000801608F10108D648784400EBC4000D9638
:1044C00090ED00BB9DED0C0B53EC1B2B51EC100B36
:1044D00002F054F99DED0C0B41EC1A0B53EC1B2B25
:1044E00051EC100B01F016FC41EC100B51EC180BC9
:1044F00053EC102B01F0CAFC41EC1C0B51EC1A0BD5
:1045000053EC1C2B01F02EFF41EC190BC1488DED33
:10451000109B7844109590ED000B4FF0005040EA4E
:10452000660000EB84408DED0A0B00F500200B9037
:104530009DED0A0B53EC1B2B51EC100B02F01EF9F6
:104540009DED0C1B53EC112B02F040F841EC100BCD
:1045500053EC102B9DED100B51EC100B01F002FFF2
:104560009DED0A0B41EC1B0B53EC102B9DED100B3A
:1045700051EC100B01F0F6FE53EC1A2B02F026F86A
:1045800053EC1B2B02F0FAF853EC1C2B01F0EAFE63
:1045900041EC1B0B53EC192B51EC190B01F0E2FE13
:1045A00041EC1A0B9C480621B0EE4A0AF0EE6A0A6A
:1045B000784400F0E9FAB0EE40CAF0EE60CA53EC7D
:1045C0001A2B51EC1A0B01F0CDFE53EC1C2B01F011
:1045D000C9FE9DED100B41EC1A0B53EC192B51EC5D
:1045E000100B01F097FB53EC1B2B01F0BBFE53ECBF
:1045F0001A2B01F08FFB9DED100B41EC1A0B53ECC5
:10460000102B51EC100B01F0ADFE41EC1C0B9FED9B
:1046100084DB53EC1D2B01F07DFB53EC1A2B01F0D6
:1046200079FB0A90CDE90A519DED0A0B53EC1D2B45
:1046300051EC100B02F0A2F853EC1C2B02F09EF888
:1046400053EC1A2B01F0C2FF9DED0A0B41EC1C0B41
:1046500053EC102B9DED100B51EC100B01F082FE72
:1046600041EC1A0B53EC192B51EC1C0B01F07AFEA8
:104670009DED0A0B41EC190B53EC102B51EC1B0B6D
:1046800001F070FE53EC192B01F044FB41EC190BC7
:1046900051EC1A0B53EC192B01F03CFB1090CDE9B7
:1046A00010519DED100B53EC1A2B51EC100B02F036
:1046B00065F853EC192B01F089FF41EC190B9FEDC4
:1046C0005A0B53EC102B9DED100B51EC100B01F01D
:1046D00049FE41EC1A0B9FED560B51EC190B53ECB4
:1046E000102B01F03FFE41EC190B9FED530B53ECE7
:1046F000102B9DED100B51EC100B01F033FE53EC21
:10470000192B01F007FB41EC100B4D48784400EBEE
:10471000C40090ED001B51EC100B53EC112B01F079
:10472000F9FA41EC190B404601F065FDCDE90A01AB
:1047300053EC192B51EC1A0B01F0ECFA41EC100B75
:104740004048784400EBC40090ED00BB51EC100BE6
:1047500053EC1B2B01F0DEFA9DED0A1B53EC112BE1
:1047600001F0D8FA0690CDE906519DED0A0B53EC05
:10477000102B9DED060B51EC100B01F0FFFF53ECDD
:104780001B2B01F0FBFF53EC1A2B01F0F7FF53EC4E
:10479000192B01F01BFF41EC100B00BF781EB0EE8F
:1047A00048AAF0EE68AA5AEA000008BF9FED268BDF
:1047B0009DED241B53EC102B8DED001B00959DED02
:1047C000240B51EC100B01F0CDFD9DED000B41ECE5
:1047D000190B53EC102B9DED240B51EC100B01F039
:1047E000CDFF9DED061B53EC112B01F0BBFD2FE01F
:1047F000FE822B654715F73F44DF5DF80BAE543E54
:1048000000000000000040438E9803007AB60B00C1
:10481000D4260000022700000C2600000000000043
:104820000000000000000840000000E009C7EE3F63
:10483000FD033ADC09C7EE3FF5015B14E02F3EBEF5
:10484000A02400005A240000000000000000F0BF77
:1048500053EC192B01F05EFA9DED060B41EC190BA0
:1048600053EC102B9DED000B51EC100B01F07AFD79
:10487000CDE910019DED100B51EC190B53EC102BF1
:1048800001F048FACDE902010C46AB498C422FDB1E
:10489000611A084318D19DED100B53EC102B9DEDC0
:1048A000020B51EC100B01F069FF41EC1B0B9FED6B
:1048B000A40B51EC190B53EC102B01F02BFA53EC19
:1048C0001B2B01F04DFE2DD20220FBF7B2FE00F0B3
:1048D0000BFA10EE901A18EE900A8DED020B8DED8A
:1048E000008B61F31E0003909DED020BFFF7EFBB01
:1048F000954A24F00041914214D39449214408433D
:104900007FF4E5AC9DED100B53EC102B9DED020BED
:1049100051EC100B01F032FF53EC192B01F020FE8B
:104920007FF6D5AC24F0004089498A4A002601EB85
:10493000205182422BDA481C4FF4801121FA00F0FA
:104940002044854AC0F30A517A44A1F2FF3192ED26
:10495000000B824A8DED0A0BCA4020EA0202C0F326
:10496000130040F48010C1F1140120FA01F60B92FB
:10497000002CB8BF76429DED0A0B53EC102B9DED39
:10498000100B51EC100B01F0F9FECDE910019DED7B
:10499000100B51EC190B53EC102B01F0BBF99FEDF0
:1049A000700B0A90CDE90A5153EC102B9DED0A0BC8
:1049B00051EC100B01F0D6FC41EC1B0B9FED6A0B88
:1049C00053EC102B9DED0A0B51EC100B01F0CAFCBF
:1049D0009DED100B41EC1C0B53EC102B9DED0A0BC5
:1049E00051EC100B01F0CAFE53EC192B01F0EEFD57
:1049F0009FED5F1B53EC112B01F0B4FC53EC1C2B0F
:104A000001F088F941EC190B51EC1B0B53EC192BFD
:104A100001F080F9CDE902019DED020B53EC1B2B57
:104A200051EC100B01F0AAFE53EC192B01F0CEFD56
:104A30009DED020B41EC190B53EC102B51EC100BBC
:104A400001F090FCCDE90A014B489DED0A0B0521D0
:104A5000784400F099F89DED0A1B51EC100B53ECD3
:104A6000112B01F07FFC9DED021B53EC112B01F08B
:104A7000ADFDCDE906019DED020B53EC192B51EC78
:104A8000100B01F06FFC53EC192B01F043F99FED73
:104A90003C0B41EC190B53EC102B9DED060B51EC2C
:104AA000100B01F06BFE9DED060B41EC1B0B53EC64
:104AB000102B9DED020B51EC100B01F053FC53EC4D
:104AC0001B2B01F0E3F953EC192B01F057FE9DED80
:104AD000021B53EC112B01F051FE53EC1A2B01F089
:104AE00075FDCDE9020101EB065001150029C8BF93
:104AF000039015DC9DED020B324651EC100B01F0DA
:104B0000C0FFFFF793F9042808BF00F0FDF8324614
:104B10009DED020B51EC100B01F0B3FFCDE902014A
:104B20009DED020B51EC180B53EC102B01F01AFC0D
:104B3000FFF72DBB000000000000904000000000C7
:104B4000FE822B654715973C00CC904000346F3FA8
:104B500001FCFFFF0000E03FCC220000FFFF0F0040
:104B600000000000432EE63F396CA80C615C20BEBB
:104B7000EF39FAFE422EE63F9C21000000000000C3
:104B8000000000000000004070B504462DED028BCF
:104B90004D1E00EBC500B0EE408AF0EE608A90ED4D
:104BA000000B35F0060017D053EC182B51EC100B0E
:104BB00001F0D8FB41EC100B6D1E04EBC50090ED2D
:104BC000001B51EC100B53EC112B01F0A3F841EC3E
:104BD000100B35F00600E7D1022D36D0042D1CD085
:104BE000062D1CBFBDEC028B70BD53EC182B51EC95
:104BF000100B01F0B7FB94ED0A1B53EC112B01F0E5
:104C000089F853EC182B01F0ADFB94ED081B53EC25
:104C1000112B01F07FF841EC100B53EC182B51ECE9
:104C2000100B01F09FFB94ED061B53EC112B01F0D0
:104C300071F853EC182B01F095FB94ED040B53EC39
:104C4000102B01F067F841EC100B53EC182B51ECD2
:104C5000100B01F087FB94ED021B53EC112B01F0BC
:104C600059F853EC182B01F07DFB94ED001B53EC2D
:104C7000112B01F04FF8BDEC028B41EC100B70BD15
:104C80009FED070B10B553EC102B9FED070B51EC6C
:104C9000100B01F0FBF841EC100B10BD0000000000
:104CA0000000000000000000000000000000F03FD5
:104CB00010B553EC112B51EC100B01F02BF841EC1B
:104CC000100B10BD000000009FED050B10B553EC5C
:104CD000102B51EC100B01F0D9F841EC100B10BD6A
:104CE00000000000000000009FED050B10B553EC24
:104CF000102B51EC100B01F035FB41EC100B10BDEB
:104D000000000000000000709FED050B10B553EC93
:104D1000102B51EC100B01F025FB41EC100B10BDDA
:104D2000000000000000001030B51A48184A03784F
:104D3000111D5B5804786FF30F0343F003036350B6
:104D4000154B134D4C330478083513496351104CFF
:104D500005780C34114B2B510378D358047843F069
:104D600001031351202393600378D358007843F054
:104D700010031350886840F001008860886840F094
:104D800080408860886840F44070886030BD0000D2
:104D9000006402400E6B0008002001404C0000201F
:104DA00010B536482DED028B816841F0804181605D
:104DB0000120FBF7EFFC9FED328B51EC100B53EC15
:104DC000182B01F0CFFA01F0E9F92F4CA080022056
:104DD000FBF7E0FC53EC182B51EC100B01F0C2FA7E
:104DE00001F0DCF9E0800320FBF7D4FC53EC182B36
:104DF00051EC100B01F0B6FA01F0D0F9E08204207A
:104E0000FBF7C8FC53EC182B51EC100B01F0AAFA7D
:104E100001F0C4F920830520FBF7BCFC53EC182BF0
:104E200051EC100B01F09EFA01F0B8F960830620F6
:104E3000FBF7B0FC53EC182B51EC100B01F092FA7D
:104E400001F0ACF9A0830720FBF7A4FC53EC182B6E
:104E500051EC100B01F086FA01F0A0F9E08300207C
:104E6000FBF798FC53EC182B51EC100B01F07AFA7D
:104E700001F094F92084BDEC028B10BD00200140AC
:104E80000000000000002440A8000020DFED0A0A16
:104E90000C4920EE200ADFED090A20EE200ADFEDA2
:104EA000080A80EE201ABCEEC10A10EE100A80B289
:104EB000086000F009B800000000C842000080450A
:104EC00000404E45180100202DE9F04318494FF6E7
:104ED000FF7606EA80004FF40055C0F30D048D61A3
:104EE0008A148A610A2000F06FFA280488610A2077
:104EF00000F06AFA00234FF400684FF00069EF03F6
:104F00008A61200401D5404600E0484688610A20B5
:104F100000F05AFA8F610A2000F056FA5B1CDBB2EF
:104F200006EA4404102BEBD38D61BDE8F08300004A
:104F3000000C0240DFED090A20EE200ADFED080A2E
:104F400020EE200ADFED070A80EE201ABCEEC10A2F
:104F500010EE100A80B200F007B800000000C8424E
:104F60000000804500404E452DE9F043184E4FF6B5
:104F7000FF7808EA80004FF48072C0F30D05B2613B
:104F8000144953008B610A2000F01EFAF701B76143
:104F90000A2000F019FAB946474600244FF000787D
:104FA0008B61280401D58A6101E0C1F818900A20BC
:104FB00000F00AFAC1F818800A2000F005FA641C13
:104FC000E4B207EA4505102CEAD3B261BDE8F083EC
:104FD00000000240000802402DE9FC410746022281
:104FE0003049FBF767FA304C012568B32D4903229D
:104FF0002F393846FBF75EFA68B32A4903222B396A
:105000003846FBF757FA002823D0264903222739D0
:105010003846FBF74FFA10B32249032223393846AA
:10502000FBF748FA0026F0B11E4903221F39384623
:10503000FBF740FA00280CD1207802282BD02078EA
:1050400003282BD0E67003E065702078062800D096
:105050002570BDE8FC81BDE8FC4100F0FBB8BDE86F
:10506000FC4100F069B811480096019601780522CC
:10507000491CC9B2017080680144684600F004FC14
:105080000849684615390522FBF714FA08B1E6709D
:10509000DFE7E570DDE7E670032001E0E57004205E
:1050A0002070D6E7856B0008400700203001002003
:1050B0000EB50B490D2201F132008DE80700A0F179
:1050C0001B0308A232210A48FBF75EF90848FBF7E8
:1050D000D2F903B0C1B206485DF804EB00F0FABAA9
:1050E000536B0008257325732573256300000000AA
:1050F000DC0600200EB50B490D2201F10B008DE8F6
:10510000070000F10C0308A232210A48FBF73CF922
:105110000848FBF7B0F903B0C1B206485DF804EBEC
:1051200000F0D8BA536B00082573257325732563E7
:1051300000000000DC0600203EB500242F4800944B
:1051400001940294816800780A220144684600F0C4
:105150009BFB012069460A5C303A092A01D80A54AF
:1051600000E00C54401CC0B20728F4D99DF801009F
:10517000234940F6354248439DF8021011FB02F1E5
:1051800000EB41109DF8031040F2712211FB02F177
:1051900000EB01109DF804109FED1A1A01EB41027B
:1051A000C2EBC11100EBC1009DF8051001EBC1027B
:1051B00002EB011100EB81009DF8061001EB81016B
:1051C00000EB41009DF80710084400EE100A9DF81E
:1051D0000000F8EEC00A2D2880EE810A01D1B1EE60
:1051E000400A09480178062901D005210170DFED48
:1051F000070A20EE200A80ED010A3EBD30010020A2
:1052000040420F000050C3474007002000007A448E
:105210000EB50B490D22C81C8DE8070000F11403E0
:1052200008A232210A48FBF7AFF80948FBF723F937
:1052300003B0C1B206485DF804EB00F04BBA0000C1
:10524000536B000825732573257325630000000048
:10525000DC0600201CB5002413480094019401785A
:105260000522491CC9B2017080680144684600F0FB
:105270000BFB0E4968460522FBF71CF90C4950B19F
:105280008C700878012805D18878002802D1012087
:1052900000F010F81CBD0120887008780628F0D0B6
:1052A00002200870EDE7000030010020706B00085C
:1052B000400700201FB50F4A0D21D31D10B102F188
:1052C0001C0001E00B482330CDE90030CDE902217C
:1052D000084B09A2173332210A48FBF755F8094851
:1052E000FBF7C9F804B0C1B2BDE81040054800F0B2
:1052F000F1B90000536B00082573257325732573DE
:1053000025630000DC0600200EB50B490D2201F1DB
:105310000F008DE8070000F1080308A232210A48B7
:10532000FBF732F80848FBF7A6F803B0C1B206480D
:105330005DF804EB00F0CEB9536B000825732573BC
:105340002573256300000000DC0600201FB50F4A0E
:105350000D2102F1130310B102F11C0001E00B4812
:105360002330CDE90030CDE90221084B08A21733E4
:1053700032210A48FBF708F80848FBF77CF804B02C
:10538000C1B2BDE81040054800F0A4B9536B000855
:10539000257325732573257325630000DC06002023
:1053A00006484FF400518161C903816104498015A9
:1053B000886104494004886170470000000C024085
:1053C000000002400008024001E0401EC0B2002878
:1053D000FBD170471E2170B5B0FBF1F2B0FBF1F5C7
:1053E00001FB120447F2305603E0304600F00EF89D
:1053F0006D1E002DF9D1002C06D04FF47A70604359
:10540000BDE8704000F002B870BD000070B54FF00C
:10541000E024002265690A49A369496A4843A169F1
:105420009942FCD002D2A3EB010302E0A5EB0106F6
:1054300033441A440B468242F1D300BF70BD0000D2
:105440000000002082B0CDE9000121F00040019071
:105450009DED000B02B051EC100B70472DE9F047A9
:105460002B4C2DED028B207801284DD104F1140234
:10547000284B20691188002523F81010E36819448F
:10548000244B8846E160143B518823F81010A36830
:105490001944204BA160283B928823F810206368B0
:1054A000401C1A446260206109282CDD0A26B2FBE8
:1054B000F6F0194F2561DFF864903880B1FBF6F003
:1054C00040F6E441484309EB1030656000F0FBFE14
:1054D0009FED138B53EC182B00F0D8FC00F05EFE10
:1054E0007880B8FBF6F040F6E441484309EB103011
:1054F000A56000F0E8FE53EC182B00F0C7FC00F0AC
:105500004DFEB882E5602570BDEC028BBDE8F087EA
:105510003800002064010020A800002024FAFFFFCA
:10552000CBA145B6F3FDB43FF0B5304C304831491E
:1055300022784FF0000316064FF0010503D5EE0563
:105540008661CB7102E080268661CD7157064FF4EB
:10555000807603D5360486618B7101E086618D719A
:1055600097064FF4007603D5360486614B7101E04F
:1055700086614D71D7064FF4806603D53604866187
:105580000B7101E086610D7117074FF4006603D5BA
:1055900036048661CB7001E08661CD7057074FF409
:1055A000805603D5360486618B7001E086618D706C
:1055B00097074FF4005603D5360486614B7001E01F
:1055C00086614D70D6074FF4804203D01204826189
:1055D0000B7001E082610D706078810705D5064A85
:1055E0000221117000F0FD006070F0BDA4000020E9
:1055F00000100240100100204007002038B50021B3
:105600000E4C00910421A06021700D4949780029B9
:1056100000F104010AD00322684600F035F9207831
:10562000C01C20706846FFF7D7FC38BD02226846D0
:1056300000F02AF92078801CF3E7000030010020F8
:1056400040070020084900220A7088600748C860A7
:105650000748086107484861074888610748C861EA
:10566000074808627047000040070020B15000085A
:1056700011520008B5520008F550000809530008FF
:105680004D530008F8B5104C2068104DC0F30010C1
:10569000002640B1206800906068009029790C488D
:1056A000FFF7ACFF6E602068C0F34010002809D0FF
:1056B0006868322800DD6E606168054A68681154C8
:1056C000401C6860F8BD000000440040300100202C
:1056D0000E070020024A93680A460146014818470F
:1056E000400700200044004070B5254C207800257C
:1056F000062828D0234E3068012823D1207878B19D
:10570000207801280FD0207802280FD02078032895
:105710000ED0207804280FD0207805280FD010E074
:10572000FFF7C6FC0DE0FFF773FD0AE0002000E084
:105730000120FFF70BFE04E0FFF7DCFC01E0062090
:105740002070356070BD104E30680128FAD1A06914
:10575000804794ED010A0D49B5EEC00AF1EE10FA4A
:1057600004DBBCEEC00A10EE100A06E0B1EE400AFF
:10577000BDEEC00A10EE100A40420881E1E70000C9
:10578000400700207C0000205C000020A8000020D2
:10579000384C00262670FBF7C3FAFEF7ADF8FCF78D
:1057A00085FCFCF737FCFCF715FEFCF7FDFEFDF76A
:1057B00015F8FCF767FBFCF79BFDFDF7A7F8FCF776
:1057C000BBFDFCF729FFFCF77FFFFCF765FEFCF74C
:1057D00025FE2948016841F001010160C16841F0DE
:1057E0000101C160416C41F400414164234F244DEB
:1057F00028680128FCD1207840B1012812D0022865
:1058000023D00328F4D100F05BF9F1E71D494FF4F0
:1058100080008861FDF70AFD16480821283000F055
:1058200057FA1FE03878012802D13879012809D0C9
:1058300010480821303000F04BFA2078401C2070CE
:105840002E60D5E70120A060F7E73878022802D162
:10585000387902280BD007480821303000F038FA98
:1058600000F018F92E602078401C2070C0E702205C
:10587000A060F5E70000002000040040280600209A
:10588000840000200010024004E000BF11F8013B3A
:1058900000F8013B521E92B2F8D2704710B5114881
:1058A00040F2FF34024683880F491268A34205D3B1
:1058B000002383801360EE20486010BD49680B4CC4
:1058C0002170D1548188491C81800948016821F0E8
:1058D0000101016000214162016841F001010160A4
:1058E00010BD000068060020004800408C00002029
:1058F00000140040074A002102F5886002608180A0
:10590000C1800172C2604FF480620282418202480B
:10591000FCF7AAB92802002000480040094810B549
:10592000C3780748064C0C30195003212046FBF77A
:10593000DBFE2046BDE810400321FBF7C1BE00009E
:1059400000600240336B000870B509486FF0010138
:105950000161016821F001010160064C0025A08869
:10596000E080A58001202072FDF710F9257270BD3E
:1059700000140040680600200448C16841F001019D
:10598000C160016841F001010160704700140040EE
:1059900010B50A4C2078032801D901202070FDF7AA
:1059A0005FFCA0680A2190FBF1F1054A207802EB28
:1059B0004002401C9181207010BD00001C0100209D
:1059C000A800002070B586B00D4606461446142186
:1059D0006846FAF7FFFD8DF8006003208DF801009E
:1059E000280A8DF80200200A8DF804008DF8035073
:1059F0008DF8054006216846FDF75FF88DF8060032
:105A0000000A8DF807000821684600F061F906B029
:105A100070BD022211460120FFF7D4BF02223A21B5
:105A20001046FFF7CFBF00B52DED048B83B041ECDE
:105A3000190B00F0D7FD41EC180B18EE100A18EE08
:105A4000901A8DED008B002818BF0120084320F02C
:105A50000040C0F17F6000F1E040C00F14D019EEAB
:105A6000101A19EE900A8DED009B002918BF012134
:105A7000084320F00040C0F17F6000F1E040C00F1B
:105A800004BF0120FAF7D5FD51EC180B03B0BDECB3
:105A9000048B00BD10B5FAF71DFFFEF783F9FFF781
:105AA0007FFCFFF769FFFFF725FFFFF73DF9FCF7E4
:105AB000C9F9BDE810400148FFF7C4BDA55C000866
:105AC00070B5564D574C584E2DED028BF3EE098AAA
:105AD00028889FED538A00EE100AF8EE400A80EE07
:105AE000880AD4ED040AB4EE600AF1EE10FA11D07F
:105AF00000EE100AF8EE400A80EE880A10EE100A56
:105B000084ED040AB04201DDC4ED048A94ED040A78
:105B1000FFF7BCF9688800EE100AB8EE400AC0EE44
:105B2000080A94ED050AF4EE400AF1EE10FA11D0DD
:105B300000EE100AF8EE400A80EE880A10EE100A15
:105B400084ED050AB04201DDC4ED058A94ED050A35
:105B5000FFF7F0F9FFF724F9FFF71AFFFFF7C4FD8D
:105B6000FFF77CFCFFF7E0FC304E307800F00400DB
:105B7000E060FEF723F96080C14371706FEA102086
:105B80003070E16800F04000884208D0A8884FF6E5
:105B9000DC71401C80B2A880884200D9A980244EC4
:105BA0003068012815D1A068224D012814D00228A0
:105BB00023D0E978A879C1EB0161084429796A7991
:105BC000C1EB0141C2EB02221144084420620020D3
:105BD0003060BDEC028B70BDFFF71BFFE978A87940
:105BE000C1EB0161084429796A79C1EB0141C2EB3B
:105BF000022211440844A061E9E7FFF70FFFE978AA
:105C0000A879C1EB0161084429796A79C1EB0141A6
:105C1000C2EB022211440844E061D8E7DA00002018
:105C200000007A44000000200000C841A6000020C7
:105C3000640000202806002030B5174800F10C0150
:105C400051E8002F42F0100241E80023002BF7D169
:105C50001349114A114D121D8C7908350F4B6251B1
:105C600000F1140252E8004F44F0800442E800457D
:105C7000002DF7D18A799A58897942F010025A504A
:105C800010F10C0050E8001F41F0200140E8001224
:105C9000002AF7D130BD00000044004000600240FF
:105CA0007D6B0008094810B583790748064C0C3015
:105CB000195006212046FBF717FD2046BDE810408D
:105CC0000621FBF7FDBC000000600240336B0008BA
:105CD000094A10B59379074A064C0C3298500A4687
:105CE00006212046FBF700FD2046BDE810400621B6
:105CF000FBF7E6BC00640240336B000881F0004112
:105D0000704780F00040704721F00041704720F05C
:105D10000040704710B591EA030F48BF83F000437D
:105D200000F13485841A71EB030C05D2121943EB90
:105D30000C03001B61EB0C01DFF824E14FEA115466
:105D4000A4EB135C1EEA430F18BF9EEA445F73D0B6
:105D500023EA0E03DCF1200E21EA045143F4801300
:105D600032D322FA0CFE10EB0E0023FA0CFE41EBAC
:105D70000E01CCF1200E03FA0EFE10EB0E0051F1D5
:105D80000001B1F5801FCCF1200E32D201EB04519D
:105D900012FA0EF2BDE8104058BF7047401C38BFE1
:105DA0005FEA420218BF7047002814BF20F00100CC
:105DB00041F100014FEA410313F5001F38BF70475E
:105DC000A1F1C04100F0C6BB012A43EB0302ACF1D4
:105DD000200CDCF11F0E32BF4FF0000E23FA0CF343
:105DE00010EB030041EB0451B4EB115FD0D0A1EBF9
:105DF000045101F5801149085FEA300001EB0451BC
:105E00000ED350F1000038BF12FA0EFE08D1BDE8E3
:105E10001040C9E7401C38BF5FEA4202CAD1C3E75D
:105E2000BDE810404FEA410313F5001F38BF70472B
:105E3000A1F1C04100F08EBB9EEA445F08D011EA98
:105E40005E0FBDE8104004BF01F000410020704724
:105E5000BDE8104070B500F02FFB00BF64FBBE3EF4
:105E60000000E0FF02494FF0000000F0D8BD00BF85
:105E70000000F87F491058BFC1F140415B1058BF86
:105E8000C3F140438B42EFF3008070472DE9C041DE
:105E900030B4DFF8A0C23CEA111418BF3CEA131476
:105EA00000F0EC8081EA03051CEA111444EAD57481
:105EB00018BF1CEA131500F0C780A4EB05044FF0CF
:105EC000004545EAC12145EAC32341EA505143EA6E
:105ED000525304F17F74994204F500344FEAC02014
:105EE0004FEAC22208BF904200F09C804FEA13653F
:105EF0000FF24016765D4FEA134506FB05F7C7F132
:105F0000807706FB07F74FEAD737A7FB036876428F
:105F1000C8F58038A7FB06CE38BFA8F1010807FBFB
:105F200008E64FF0000EA6FB028CE6FB03CEDCF188
:105F3000000CCEF1004E38BFAEF1010EA6FB0C589E
:105F40004FF000074FF00005E6FB0E87A1FB08C6E7
:105F5000A0FB07CE16EB0E0645F10005E1FB076539
:105F600015F1E04E7EBFA4F580345FEA46066D4130
:105F700016F1800745F100054FEA17274FEA06663C
:105F800047EA0567A6F1DE46B6F1805F4FEA1525C0
:105F90001FD9384624F0010C05EBC471BCF1FE6F2B
:105FA00001EB0C1102D8F0BCBDE8008124425CBFBB
:105FB00001F5801E9EEAC47F02D4F0BCBDE80081DA
:105FC000244238D4F0BCA1F1C041BDE8004100F04A
:105FD000C1BA4FEAD22242EA43524FEAD323A7FB87
:105FE00002864FEAD02040EA415007FB03661EEAD2
:105FF0000E0F4FEAD12105FB026658BFA6EB0056F3
:10600000B6EB00564FEA520E4EEAC37E18EB0E0E68
:1060100056EB530EBDD518EB02085E417F1C55F1BF
:106020000005B6E74FF480154FF000074FF000066B
:106030004FF00008ADE7F0BC4FF0000001F1C041A7
:1060400001F00041BDE8008111EA0C1F0CEA1315B4
:1060500000D00CE013EA0C1F00F025804FF0000088
:10606000F0BC81EA030101F00041BDE80081F0BC11
:10607000BDE8004181EA030100F06CBAF0BCBDE864
:10608000004170B500F018FA097EFC3E00F007B838
:1060900081EA03014FF0000001F00041704781EAFE
:1060A000030100F057BAF0BCBDE800414FF000001A
:1060B00021497047FFFDFBF9F7F5F4F2F0EEEDEB47
:1060C000E9E8E6E4E3E1E0DEDDDBDAD8D7D5D4D3F6
:1060D000D1D0CFCDCCCBCAC8C7C6C5C4C2C1C0BF42
:1060E000BEBDBCBBBAB9B8B7B6B5B4B3B2B1B0AF48
:1060F000AEADACABAAA9A8A8A7A6A5A4A3A3A2A12C
:10610000A09F9F9E9D9C9C9B9A99999897979695E6
:1061100095949393929191908F8F8E8E8D8C8C8B82
:106120008B8A89898888878786858584848383820A
:10613000828181800000FF070000F87F4FEA410361
:106140004FEA5353A3F58063D3F11E03C8BFD3F1C5
:10615000210C0CDD4FF0004242EAC12242EA5052CB
:1061600032FA03FC8CEAE17CACEBE1707047102B57
:10617000C4BF0020704703F5787CBCF1FF3F04D01A
:106180006FF0004282EA2100704770B500F094F988
:106190004992248000207047F2E700004FEA115333
:1061A000A3F58063D3F11E03A8BFD3F1200C08DB55
:1061B0004FF0004242EAC12252EA505232FA03F052
:1061C000704709420BD4102BC4BF0020704703F561
:1061D000787CBCF1FF3F05D04FF0FF3070474FF0A7
:1061E0000000704770B500F067F900BF4992248045
:1061F00000207047F0E710F0004248BF4042B0FA7C
:1062000080F310FA03F10AD0C3F11D0303F5806394
:106210004FEA415002EB035202EBD12170474FF09D
:10622000000070477FEAE17202D1101A62EB0101AF
:10623000B1FA81F30B3B24D3994012D1B0FA80F329
:1062400010FA03F108BF7047C3F11D0303F5406363
:1062500003EBC2234FEAD1224FEA415002EB035134
:106260007047C3F1200C20FA0CFC9840C3F13203B4
:1062700003F5406303EBC22341EA0C0101EB035138
:10628000704710B5C3F1320CC3F10004C4F1200E05
:106290000CF5406C0CEBC22201FA0EFC21FA04F161
:1062A00000FA0EF3E040BDE8104040EA0C0001EBBC
:1062B000025138BF7047401C41F100015B0008BF2C
:1062C00020F001007047B0FA80F310FA03F10AD011
:1062D000C3F11D0303F580634FEA41504FEA0352B7
:1062E00002EBD12170474FF00000704751EA030CD8
:1062F00017D41CF5801F58BFBCF5801F00F1068025
:10630000994218BF704708BF9042704707D711F5F0
:10631000801F58BF13F5801F19D4994270478942D6
:1063200070471CF5801F08D5BCF5801FF7D58B4240
:1063300018BF704708BF824270474FF4001C1CEB27
:10634000410F38BF1CEB430F01D28B42704770B531
:1063500000F0B2F8922449004FF000514FF0805302
:10636000FFF788BDDFF848C170B51CEA111E1EBFDB
:106370001CEA13159EEA0C0F95EA0C0F00F06F80D3
:1063800081EA030423EA4C134EEAD47E21EA4C113D
:1063900041F4801143F48013AE44A1FB024CA0FBF6
:1063A0000365AEF17F7E361955EB0C05A1FB034C5E
:1063B0004CF10003A0FB021C16EB0C06654153F1E7
:1063C0000003094218BF46F0010613F4007F0BD109
:1063D0004FEA03314FEA0530340341EA155140EAF0
:1063E00016506FF003020AE04FEAC3214FEAC520BE
:1063F000F40241EA555140EA56506FF0020202EBB6
:106400002E4201EB025585EACE710AD05FEA440CB8
:1064100018BF24F0004450F1000041F1000120EACF
:10642000D47040F2FE7C624500D270BDA84214BF19
:106430004FF080444FF04044002E08BF0024BEF1CE
:10644000806FA8BFA1F1C041BDE8704080F282809A
:106450004FF0000001F1C04101F0004170479EEA99
:106460000C0F0CEA131518BF95EA0C0F06D04FF06D
:10647000000081EA030E0EF0004170BD00F01CF830
:106480008900013E00F007B800F009B84FEA430C5C
:106490005FEA5C5C08D081EA030100F05BB84FEA78
:1064A000410C5FEA5C5CF6D14FF000000149704797
:1064B0000000FF070000F87F0EF1020E2EF0030E21
:1064C0005EF8046B364205D4012A43EB030515F54B
:1064D000001F12D8012841EB010C1CF5001F0CD83D
:1064E0000ED14FEAD17C15F5001F0CEB4C0C0CF1D2
:1064F000020C08BF4CEBD37C04E04FF0080C01E029
:106500004FEAD37C0CEB4C0526FA05F606F007069D
:10651000B6F1040C06D20EEB860CBDE870404CF0D0
:10652000010C6047DFE80CF0090B02024FF000415C
:106530004FF00000A1F5002170BD1946104601285A
:1065400051EB010418BFD4F5001484BF002001F002
:10655000004170BD0808A0F500114FEA31017047F5
:1065600053EA010C17D41CF5801F58BFBCF5801FDF
:1065700000F106808B4218BF704708BF8242704707
:1065800007D713F5801F58BF11F5801F19D48B4210
:1065900070479B4270471CF5801F08D5BCF5801FD3
:1065A000F7D5994218BF704708BF904270474FF423
:1065B000001C1CEB430F38BF1CEB410F01D299426A
:1065C00070470FB40CBC03BCFFF7C1BE91EA030FC8
:1065D00010B581F000413FF5A5AB83F0004300F01A
:1065E000D5B800002DE9F04101F5801CBCF5001F75
:1065F000C0F2A9804FEA115C21EA0C510CF1FD0CAC
:1066000041F480115FEA5C0C0CF5C07C01D34000C2
:10661000494130A4890241EA905187028E0E0A0C4A
:10662000A45D04FB04F602FB06F6C6F14046A4FB9B
:106630000662F60D46EA422606FB06F4A4FB012399
:106640005242C3F1404338BF5B1EA6FB0242002406
:10665000E6FB0324D20B42EA4446A6FB0623A1FB39
:1066600002E2A3FB07E4E3FB61426442C2F1404E55
:1066700038BFAEF1010EA6FB04234FF00002E6FB8B
:106680000E32A2FB03463400E2FB6264A1FB06E685
:10669000A4FB07E8E4FB61687642C8F1405838BFC4
:1066A000A8F10108A2FB06E4A3FB08E5E2FB68549D
:1066B000A1FB05E6A7FB04E8E1FB648618F12005D1
:1066C00056F10006A809A8F11B08B10908F03F0817
:1066D000B8F10A0F40EA86601CD901EB0C51BDE805
:1066E000F08100BFFCF5EEE8E2DDD8D3CFCBC7C325
:1066F000C0BDB9B6B4B1AEACA9A7A5A3A19F9D9BDF
:106700009A9896959392908F8D8C8B8988878685A1
:1067100084838281A0FB006800FB01F208EB420841
:10672000B8EB872807D5341858EB0104D5D5401CA1
:1067300051F10001D1E7341A78EB0104CDD4401EA9
:1067400071F10001C9E75FEA4C0C5FEA9C5C0DD176
:1067500005D34FF0000001F00041BDE8F081BDE835
:10676000F04170B5FFF7A8FE6DDBFFBEBDE8F0415C
:106770004FF00000004970470000F87F10B591EA23
:10678000030F48BF83F000433FF5CCAA841A71EB96
:10679000030C07D212198CF0004C43EB0C03001BC6
:1067A00061EB0C01DFF8A4E14FEA1154A4EB135C98
:1067B0001EEA430F18BF9EEA445F00F0B08023EA50
:1067C0006E03524221EA0451C3EB6E0338BF5B1ED5
:1067D000DCF1200E25D322FA0CFE10EB0E0043FA5A
:1067E0000CFE41EB0E01CCF1200E03FA0EFE10EB75
:1067F0000E0051F10001CCF1200E29D412FA0EF254
:1068000001EB0451BDE8104058BF7047401C1CBF4D
:10681000B2F1004F704700280CBF491C20F0010066
:10682000704712EB020E43EB030218BF4FF0010E4C
:106830004EEA4202ACF1200CDCF11E0E54D943FAB0
:106840000CFE10EB0E0051F1FF31CCF11E0ED5D530
:106850000EF1010E12FA0EFE404141EB010101EB77
:10686000445C5FEA5C5C10D910EBDE7001EB045114
:1068700038BFBEF1004FBDE8104018BF7047002878
:106880000CBF491C20F00100704730D24FEAD42CD5
:1068900011F5001124F400641BD0B1FA81F20B3A17
:1068A000A41AA41ED2F12003914030FA03F3194335
:1068B000904001EBCC71002C01EB0451BDE810407D
:1068C000A8BF704701F1C0414FF0000001F0004146
:1068D0007047B0FA80F310FA03F100D110BDE41A4A
:1068E000173C4805C90AE4E701EB045110BD491003
:1068F00001EB0451BDE810404FEA300002E04FF0D8
:10690000000170474A0008BF0042F8D0B2F5001FEE
:1069100028BF704701F000414FF0000070479EEA29
:10692000445F07D011EA5E0FBDE8104004BF0021AC
:1069300000207047BDE8104070B5FFF7BDFD00BFF7
:1069400040DFF63E83F00041104670470000E0FF54
:106950004FF04070E1EE100A704700004FEAC1238B
:106960000A1543EA50534FEAC02C18BF43F00043C6
:106970001BD4A2F24E02D2F57C7240F34280502A20
:10698000A8BF502223FA02F12CFA02F0D2F1200221
:1069900060B403FA02F588BF2843C2F1000223FA6B
:1069A00002F598BF284360BC704702F57C7212F56F
:1069B000826F08BF23F00043D2F12E0221DB1AD0F0
:1069C000502AA8BF502223FA02F12CFA02F0D2F189
:1069D000200260B403FA02F588BF2843C2F1000226
:1069E00023FA02F598BF284360BC4042C1F1000180
:1069F00038BF491E70479CF0000F08BF93F0004F4E
:106A0000DED070B5FFF758FD9224498000214FF089
:106A1000000070476FEAE17080F0004170470CF0B1
:106A20000F03092B08BF082000F059800A2B0BD058
:106A3000082B18BF704708BF1CF0400F0AD04FF05A
:106A400000004FF0000170471CF0400F18BF4FF0DE
:106A5000004070471CF0100F08D020F0704300F089
:106A60007F4242EAD3014FEA4370704700F0604032
:106A700021F07F4242EA000201F07F4040EA72705A
:106A800070474FF0FF0C4CF4E06C1CEA11531CBF34
:106A90009CEA030C9445C2BFDA4201EB02517047F5
:106AA000002B0DD0BCF1000F0FD0002A01F00041E7
:106AB000A4BF41F0E04141F07F614FF0000070471A
:106AC00001F000414FF00000704750EA01334FF0F1
:106AD0009B0C18BF4CF0806C7FF4C4A970471CF469
:106AE000801F11D01CF4E02F03D06FEACC31490095
:106AF00070474FF04050EFF3008222F0704242EABC
:106B0000000282F3008870474FF0000070471028A1
:106B100040587088A0B80000000004040400000879
:106B20000000000800020406080A0C1028405870F3
:106B300088A0B8102840587088A0B8000000000055
:106B4000000000010203040607080900000000011C
:106B50000203042A2A00524C5200574C5200524D54
:106B60004400525A5300575A530025303123002B0A
:106B70003030303031002B30303030300010284091
:106B8000587088A0B857435352303330303100002A
:106B9000000000000000F03F000000000000F83F8F
:106BA00000000000000000000000004003B8E23FC9
:106BB000000000000000000006D0CF43EBFD4C3E7B
:106BC000033333333333E33FFFAB6FDBB66DDB3F70
:106BD0004D268F515555D53F01411DA96074D13FB8
:106BE00065DBC9934A86CD3FEF4E454A287ECA3FB2
:106BF0003E5555555555C53F93BDBE166CC166BF34
:106C00002CDE25AF6A56113FF16BD2C541BDBBBE2C
:106C1000D0A4BE726937663E00000000000000008C
:106C2000406C0008000000203C010000C401000886
:106C30006C6C00083C0100208C0C00000002000875
:106C400001292D010300010001D5CA0203008104BE
:106C50005D01D411420192104324F4072FAA00557C
:0C6C6000AAAA55053F9001D007022001B0
:040000050800018965
:00000001FF
